:020000040800F2
:10000000E010002005010008633800082D290008D1
:1000100061380008410F0008CD61000800000000B1
:10002000000000000000000000000000E947000898
:10003000EB1A000800000000C13D0008E94A000872
:100040001F010008C13B00081F0100081F01000834
:100050001F0100081F0100081F0100081F01000800
:100060001F0100081F0100081F0100081F010008F0
:100070001F0100081F010008AD1500081F0100083E
:100080001F0100081F010008410700081F010008A8
:100090001F0100081F0100081F0100081F010008C0
:1000A000594B0008394C00081F0100081F010008C7
:1000B0003D4C00082D4F0008895100081F01000821
:1000C0001F0100081F0100081F0100081F01000890
:1000D0001F010008C55C00081F0100081F0100087F
:1000E0001F0100081F0100081F010008DFF810D0E1
:1000F00000F0E8FA00480047A9720008AFF300805A
:10010000E01000200648804706480047FEE7FEE76B
:10011000FEE7FEE7FEE7FEE7FEE7FEE7FEE7FEE7B7
:10012000094B0008ED0000082DE9F0410024061BF2
:10013000254671F1000605DA01240027D0EB0700FF
:1001400067EB0101161E73F1000605DA0027D2EBFA
:100150000702012567EB030300F0D0F986460E463F
:1001600017469C46AC4204D00025D0EB050E65EB4B
:10017000010624B10020D2EB000760EB030C7046AF
:1001800031463A466346BDE8F08140EA01039B07E9
:1001900003D009E008C9121F08C0042AFAD203E0FC
:1001A00011F8013B00F8013B521EF9D2704780EA7A
:1001B000010210B502F00043400022D04A001FD0D7
:1001C000010E01EB1261C0F35600C2F3560240F477
:1001D000000042F40002A0FB022000047F39140456
:1001E00000D0401C50EA124001D44000491EC2B267
:1001F0000C0604EBD010401C4008802A02D003E01B
:10020000002010BD20F00100002900DA0020184372
:1002100010BD2DE9FE4F81EA030404F0004421F0F3
:10022000004100944FF0000B23F0004350EA01041A
:100230005ED052EA03045BD0C3F30A54C1F30A55FB
:100240002C44A4F2F3340194A0FB0254C1F3130133
:1002500041F48011C3F3130343F4801301FB024400
:1002600000FB034E840A970A44EA815447EA835705
:10027000A4FB076802958D0A05FB07854FEA932CBE
:1002800004FB0C542705029D4FEA065847EA16372F
:10029000B5EB08056EEB070C870E920E47EA811747
:1002A00042EA8312A7FB0201B6EB0B0164EB0004E8
:1002B0002B0D43EA0C335E1844EB1C50DA465146D2
:1002C000E7FB0201C5F313044FEA0B3343EA14536F
:1002D0004FEA0432019C43EA0603A4F10C040294A1
:1002E000009CCDE900B400F09FF903B0BDE8F08FA9
:1002F00000200146F9E72DE9F04D81EA030404F0FE
:10030000004B21F0004514464FF0000A23F0004155
:1003100050EA050220D054EA01021DD0C5F30A5765
:100320000246C5F31303C1F31300C1F30A5640F4A8
:10033000801543F48013A7EB0608101BD64608F27D
:10034000FD3873EB050002D308F1010801E09218B3
:100350005B41B8F1000F03DA00200146BDE8F08DE3
:1003600000204FF48011064684460EE0171B73EB05
:10037000050705D3121B63EB050306434CEA010C8A
:1003800049084FEA300092185B4150EA0107EDD16D
:1003900052EA030012D082EA040083EA050108430E
:1003A00005D0101BAB4106D20122002306E000223B
:1003B0004FF0004302E06FF0010253101AEB060009
:1003C0004CEB085110EB0A0041EB0B01BDE8F04D7E
:1003D00000F01BB970B521F0004303430CD0C1F30A
:1003E0000A550024D5EB040564EB0403D617AD1AB7
:1003F000B34102DB0020014670BD201841EB0251E1
:1004000070BDC10F80EAE0700844CA07962300213E
:1004100000F0CDB896230022114600F0C8B80EB502
:10042000C10F80EAE0700844CA07002140F233435C
:100430008DE80E000A460B4600F0F6F803B000BD4A
:100440000EB540F2334102910021CDE900110A4678
:100450000B4600F0E9F803B000BD00F0004220F0C8
:100460000040C10DC0F3160040F400007F2901DAFE
:1004700000207047962903DCC1F19601C84001E0D5
:1004800096398840002AF4D04042704770B5C1F3D5
:100490000A5201F000450024C1F3130140F2FF337A
:1004A00041F480119A4201DA002070BD40F23343DA
:1004B0009A42A2F2334203DC524200F05FF800E0BD
:1004C00090402C43F1D0404270BDC1F30A5210B5A8
:1004D000C1F3130140F2FF3341F480119A4201DA73
:1004E000002010BD40F233439A42A2F2334203DCB3
:1004F000524200F043F810BD904010BD2DE9F05F6E
:100500000546002092469B46884606468146402482
:100510001BE0284641464746224600F02FF8534646
:100520005A46C01A914110D311461846224600F08F
:1005300016F82D1A67EB01084F46224601200021CC
:1005400000F00DF817EB00094E41201EA4F1010444
:10055000DFDC484631462A464346BDE8F09F202A64
:1005600004DB203A00FA02F1002070479140C2F10A
:10057000200320FA03F3194390407047202A04DB3C
:10058000203A21FA02F00021704721FA02F3D0400C
:10059000C2F1200291400843194670470029A8BFC4
:1005A0007047401C490008BF20F00100704710B49C
:1005B000B0FA80FC00FA0CF050EA010404BF10BC51
:1005C000704749B1CCF1200421FA04F411FA0CF17E
:1005D00018BF012121430843A3EB0C01CB1D4FEAB7
:1005E00000614FEA102042BF002010BC704700EBB2
:1005F000C35010440029A4BF10BC7047401C4900E0
:1006000008BF20F0010010BC704710B5141E73F134
:10061000000408DA401C41F1000192185B411A43C2
:1006200001D120F0010010BD2DE9F04D92469B460E
:1006300011B1B1FA81F202E0B0FA80F220329046B4
:10064000FFF78DFF04460F4640EA0A0041EA0B011E
:1006500053465A46084313D0114653EA010019D0B5
:10066000C8F140025046FFF789FF05460E46504646
:1006700059464246FFF773FF084305D0012004E0C6
:1006800020463946BDE8F08D0020054346EAE07675
:100690002C4337430A986305E40AA0EB08000022C4
:1006A000FD0A44EA47540A3002D500200146E9E732
:1006B000010510196941DDE9084500196941BDE8E6
:1006C000F04DA2E7064C074D06E0E06840F001035C
:1006D00094E8070098471034AC42F6D3FFF70AFDC0
:1006E000249500084495000870B58C1810F8015B3B
:1006F00015F0070301D110F8013B2A1106D110F8BB
:10070000012B03E010F8016B01F8016B5B1EF9D1BE
:100710002B0705D40023521E0DD401F8013BFAE744
:1007200010F8013BCB1A921C03E013F8015B01F8AF
:10073000015B521EF9D5A142D8D3002070BD000044
:1007400070B54E4C4FF490652946204600F019FADA
:10075000002864D02946204600F0A6F848490888B9
:10076000401C08800121204600F0EAFA454942F287
:100770001072B1F85000904202D2401CA1F8500013
:1007800006F06EFF404DB5F91410B5F9120005F0F2
:100790005FFE3E4CA5F84E002080A16820468847A9
:1007A000A088A5F8500003F0C5F807F05BF8384EB4
:1007B000384C3078082833D045F6AC30606042F6CB
:1007C000EF60A06042F2C400E0603348008A2080FD
:1007D000208E6080A16B2F488847208E69882F4C1F
:1007E00008444FF6FF7101EA80006886207A4FF0D6
:1007F000000540071DD501F007FB294949F6A24035
:100800000880284840F21A62C188491C89B2C18018
:10081000914204D3A16821F00401A160C58070BD9C
:1008200041F2130060604FF48060A06040F61B50FE
:10083000CAE730780A281BD2DFE800F01A0616054E
:100840000A050D1A1114EAE7BDE8704005F0A4BFCF
:1008500007F024FF08E0BDE8704002F0B5BD06F0E7
:1008600015FB01E007F056F9BDE8704007F052B9FA
:1008700000F0FEFB84F8B65070BD0000002401407B
:10088000F80600203C010020600000201407002032
:10089000EF060020D0000020EC010020980200208C
:1008A000442C0140200900206FEA112101607047AB
:1008B0000029816802D041F0010101E021F001012D
:1008C000816070470029816802D041F4807101E0A5
:1008D00021F48071816070472DE9F041824E92B021
:1008E000304600F00BF90BA800F039FA01214FF463
:1008F000C06003F01BFB00248DF831404FF46020F2
:10090000CDE90D044FF4A0204FF009080B9001270A
:100910008DF83C808DF830700BA9304600F080F9DE
:10092000724D8DF831408DF830708DF83C700BA908
:10093000284600F075F901231A460F21304600F0D1
:10094000C0F9022201231146304600F0BAF9012312
:1009500003220021304600F0B4F901230422194695
:10096000304600F0AEF9012305220B21304600F09D
:10097000A8F9012306220421304600F0A2F9012340
:1009800007220821304600F09CF9012308220321A8
:10099000304600F096F9012309220A21304600F082
:1009A00090F90121304600F084F90121284600F039
:1009B00080F901231A460521304600F055F901233C
:1009C0001A460621284600F04FF90021304600F073
:1009D000CBF84FF4E041284600F0C6F8012130463C
:1009E00000F0B8F80121284600F0B4F801213046A3
:1009F00000F0A6F80121284600F0A2F801213046B7
:100A000000F09EF90121284600F09AF940F61451B1
:100A1000374804F090FE12208DF8400002208DF837
:100A200041008DF842408DF8437010A802F046FF57
:100A300001224FF49061304600F0E8F80121304681
:100A4000FFF740FF01213046FFF732FF0121284622
:100A5000FFF72EFF304600F06EF9304600F09FF8A9
:100A60000028FAD1304600F075F9304600F082F8DF
:100A70000028FAD1284600F05EF9284600F08FF8E9
:100A80000028FAD1284600F065F9284600F072F8EF
:100A90000028FAD10121084603F024FA154D284612
:100AA00000F0C0FD684600F068FE0F4801A94C3018
:100AB0000090114881E811018020CDE904404000F8
:100AC000069080000790202008904FF44050CDE918
:100AD00009046946284600F033FE0121284600F04B
:100AE00095FD12B0BDE8F0810024014000280140CE
:100AF000002C014008000240A80200200D4910B55A
:100B0000884202D1012144150AE00B49884202D1F2
:100B10000121041504E0094988420AD10121CC03CE
:100B2000204603F00FFA2046BDE81040002103F0F4
:100B300009BA10BD0024014000280140003C0140DA
:100B40000029816802D041F4801101E021F4801174
:100B5000816070470029816802D041F4004101E0C2
:100B600021F4004181607047826822F4E0420A4328
:100B700082607047014600208968490700D501203E
:100B8000704710B50246002054680B0AC9B20C40E9
:100B90001168194202D0002C00D0012010BD01467E
:100BA00000208968090700D50120704738B5012168
:100BB0001C2003F0BBF9FF20ADF8000000248DF8E5
:100BC000034003258DF8025069460D4801F01EFBD5
:100BD0000120ADF800008DF803408DF80250694601
:100BE000084801F013FB2320ADF800008DF8034006
:100BF0008DF802506946044801F008FB38BD00003A
:100C000000080140000C014000100140002A426829
:100C1000C9B201D00A4300E08A4342607047000035
:100C200010B542680E4B0C791A400B6842EA042258
:100C30001343436083680B4A1340D1E902422243C5
:100C40004C7943EA44031A438260C26A097C22F465
:100C50007002491EC9B242EA0151C16210BD0000D2
:100C6000FFFEF0FFFDF7F1FF70B5072409290AD94F
:100C7000C568A1F10A0606EB4606B440A543B34099
:100C80001D43C56007E0056901EB4106B440A5437B
:100C9000B3401D430561836BC3F30154121B921CC7
:100CA00002EB82041F22A2409343A1400B438363C3
:100CB00070BD826B491E22F4401242EA01518163E9
:100CC000704770B5072409290AD9C568A1F10A0639
:100CD00006EB4606B440A543B3401D43C56007E09C
:100CE000056901EB4106B440A543B3401D430561CE
:100CF0001F23072A09D2446B521E02EB8202934043
:100D00009C4391400C43446370BD0D2A09D2046B8F
:100D1000D21F02EB820293409C4391400C43046338
:100D200070BDC46A0D3A02EB820293409C4391402D
:100D30000C43C46270BD816841F008018160704756
:100D40000029816802D041F4A00101E021F4A00152
:100D500081607047816841F0040181607047002123
:100D60000160017141718160C160012101747047AE
:100D700070B51E4C214694F83800B1F84250062850
:100D80001ED9B4F84A10B4F84C00A1EB000202F1ED
:100D90000902122A04D8FFF753FB0022144B0AE081
:100DA000884204D2FFF74CFB0022124B03E0FFF70E
:100DB00047FB0022104BFFF72CFAFFF786FB09E0F8
:100DC00005D12846FFF73CFB0C4A0D4BF3E70D49D4
:100DD00051F82000C5EB45116063B0EB410F03D91A
:100DE000C5EB45104000606370BD00003C0400206E
:100DF00000003440000033400000354067666666FE
:100E000066E64B40CC8C000810B50C4C20784007AF
:100E100013D5FFF7ADFF0A49A08E08800848303887
:100E2000018821F010010180001F018841F01001AC
:100E30000180207820F00400207010BD3C040020C8
:100E400040040040F0B4184816494FF49677436CBC
:100E500008468A68046815485FEAC25C42F00806E2
:100E6000007822F008054FEA047415D5002C08DB41
:100E7000120714D408B1082811D1BB420FDA8E60D2
:100E800007E012070BD508B1082808D1BB4206DAE3
:100E90008D60F0BC05F0FEBD002CF2DAE8E7F0BC96
:100EA00070470000980200203C010020EF0600205F
:100EB00070B506464089204B204C4FF480710025C8
:100EC00080B362887AB1012A0CD1E188491C89B2C9
:100ED000E1803289914205D36580E580FF2801D009
:100EE000401E708170BD70882288904201D9012215
:100EF00000E00022184601F012FA7088B18801441F
:100F00002088401C80B220808142EBD82580A088B8
:100F1000401C80B2A080F1888842E3D30120608029
:100F2000A58070BDFFE70022184601F0F8F9A58002
:100F3000E58025806580F4E7000C0140AC050020C9
:100F4000FEE70000FCB505464FF6FF7600200C4694
:100F5000ADF8006048F205078DF8040020E000BFFE
:100F600015F8010B8DF8040001A9084602F009F9F3
:100F7000BDF800009DF8041080EA0120ADF80000E3
:100F80005FF00000BDF800100A0402D587EA4101B5
:100F900001E006EA4101401CADF800100828F1DB31
:100FA000641EDDD26946084602F0D5F8BDF800009F
:100FB000FCBD00000246002004E000BF12F8013B27
:100FC0001844C0B2491EF9D27047000070B5144AE7
:100FD00085B010880024134901940094039420469E
:100FE0000494138807E00D8B009E35440095CD8B4B
:100FF000019E3544019515889D42F4D0401CC0B235
:101000008028EED3009841110748418084800198E0
:101010004111064881830183818205B070BD0000C3
:10102000F806002098020020C6050020B404002025
:1010300030B50E4902880A800C4A4388083A13806A
:101040000B1F808818802024151F2C800020401C36
:1010500080B27328FBD341F21110088044F6480097
:10106000108047F2480018802C8030BD202C0140B1
:10107000114944F648000880091D46F648000880DA
:10108000091D41F2111008800B48001F018841F032
:101090002001018009480021A0F86410A0F8621026
:1010A000A0F86010A0F85E10A0F85C10A0F85A102C
:1010B0000348418181827047182C0140980200202A
:1010C00060000020F0B54F4B4F480021DA7A0778D6
:1010D000802A27F001057DD31C684C4B02F01F02CB
:1010E00053F822204A4B14421A6802D042F02002E0
:1010F00001E022F02002474C1A60474E94F800C0ED
:10110000464CBCF1020FB4F9044043D1B3F808C017
:10111000CCF3C00ECCF3002CE6453BD03C4D2C3D2F
:1011200095F802C0BCF1000F04D0BCF1010F0FD044
:10113000A97033E05FEA025C30D55FEA826C2DD49F
:101140004FF0010C85F802C027F00405057025E07A
:101150005FEA025C22D45FEA826C1FD55FEA477CBB
:101160000BD447F004070770B0F802C0BCF1000FC1
:1011700006D0418027F0010707700227AF700DE00D
:101180004480002CF9DD47F001070770244FFF6A07
:101190004761F2E705704180318041811C4DC7886D
:1011A00095F846500FB9002C17DC077BAF4214D1DD
:1011B000B0F9027007F26667BC420EDC194FBF89B6
:1011C0005FEA477C09D45FEA877C06D45FEA427C09
:1011D00003D500E012E0FF0709D007785FEAC77C7B
:1011E00005D027F001070770418031804181C4801C
:1011F0000573500960F3CB221A60F0BD0570418081
:101200004181F0BDCC050020080900202C91000888
:1012100098020020EF06002010010020C6050020E3
:1012200060000020100A00202DE9F04796B000244D
:101230000C940D940E940F9472B69048816941F409
:1012400000718161816941F4806181614FF40040E6
:1012500002F03EFE8A4D00212846FFF733FB0021B5
:101260002846FFF725FB874E00213046FFF720FB7D
:10127000854F0021384600F0C9F901204FF4704134
:10128000401C8842FCD32846FFF738FCB146304664
:10129000FFF734FC384600F0C5F94FF46020CDE983
:1012A00012048DF8454001204FF004088DF84400E9
:1012B00010948DF8508010A92846FFF7B1FC012347
:1012C0001A4605212846FFF7FCFC012302220621CD
:1012D0002846FFF7F6FC0123032207212846FFF7E3
:1012E000F0FC012304220F212846FFF7EAFC3846D0
:1012F00000F098F9684600F040FA6148634E4C30BF
:101300000090CDF80C80CDE901648020CDE9044047
:101310004000069080000790202008904FF4405035
:10132000CDE909046946384600F00AFA0121284649
:10133000FFF7C8FA0121384600F068F90121284674
:10134000FFF7B6FA47F2305115941598401C1590E6
:101350008842FAD301212846FFF7F2FCADF82C4071
:10136000A04640F2DC5A4FF4007420E05046CDF81D
:1013700054801599491C15918142FAD330880D99F2
:1013800008440D9070880E9908440E90B0880F990B
:1013900008440F90F0880C9908440C9001212846CD
:1013A000FFF7CEFCBDF82C00401CADF82C00BDF8BA
:1013B0002C00A042DAD30D98354A40F3CF163348BB
:1013C0000A3006830E9941F3CF1444830F9941F3F9
:1013D000CF1383830C9941F3CF1CA0F804C0ACF564
:1013E000C05C40F2C371ACF59B7C8C450ED2A6F577
:1013F000C856363E8E4209D2A4F5C854363C8C42BB
:1014000004D2A3F5C853363B8B4203D3D18841F4B1
:101410008041D180D188490407D41E49028B21F82C
:101420005C2F428B4A80808B888000212846FFF702
:1014300049FA0021384600F0E9F800212846FFF774
:1014400037FA00214C464846FFF732FA0220C10223
:10145000401C8842FCD32846FFF750FB2046FFF78C
:101460004DFB384600F0DEF8FFF736FA0A493C201B
:10147000087062B616B0BDE8F087000000100240A8
:10148000002401400028014008000240120500200D
:10149000100A0020680C0020EC060020F0B53F4B3D
:1014A000404C93F856503E4B042D5B6C1DD0256884
:1014B00040F22D465D1B656043F6FB25B3F5FA5FF0
:1014C00033DDB3F5FA4F30DC41F6AD17A3F5FA532F
:1014D0005F4306EBA7364FF4B5777B4305EBA313C9
:1014E00075105B10C4E9065321E043F6D0171026AF
:1014F00041F26205BB4218DB44F25067BB420EDA90
:10150000A3F5645345F24C67D03B5F4306EBA73627
:10151000A66140F62476734305EB232303E042F2F1
:101520004713A361204BE36101E0C4E9066540F283
:10153000AE43936044F24C23401A1361106051682B
:10154000884202DA4942884200DC1160106844F2A5
:101550004C214843117D0841516A01445162106A8F
:10156000814200DD5062516AD069814201DB084648
:1015700000E050622062116840F2AE435943137B91
:10158000194118410144B2F91800884204DBB2F94C
:101590001600884200DC08B2F0BD000060000020A8
:1015A0003C0100201401002085EB010010B54FF430
:1015B0000054204600F0ACF8002813D00A490878FF
:1015C00040F008000870204600F014F80021074899
:1015D00000F01CF80648C17E012903D10021C17624
:1015E0000121017710BD0000660600204400024082
:1015F0000C0B0020C10002D5024908607047024967
:10160000486070470404024000000240002901685D
:1016100002D041F0010102E04FF6FE72114001607C
:101620007047000001684FF6FE7211400160002112
:10163000016041608160C1603149314A083990429E
:1016400003D1486840F00F0006E02D4A1432904262
:1016500004D1486840F0F00048607047284A2832BA
:10166000904203D1486840F47060F5E7244A3C3268
:10167000904203D1486840F47040EDE7204A503270
:10168000904203D1486840F47020E5E71C4A643278
:10169000904203D1486840F47000DDE7184A783280
:1016A000904203D1486840F07060D5E7154A111F99
:1016B000904203D1086840F00F0006E0114A14324E
:1016C000904204D1086840F0F000086070470D4A6D
:1016D0002832904203D1086840F47060F5E7094A67
:1016E0003C32904203D1086840F47040EDE7054A6F
:1016F00050329042EAD1086840F47020E5E70000DB
:101700000800024008040240406880B270470000B0
:1017100001460020CA0001D5034A00E0034A1268CE
:101720000A4200D00120704700040240000002403D
:10173000002A026801D00A4300E08A430260704731
:1017400030B5036847F6F07293430C6A8A68224307
:10175000D1E904452C4322438C692243CC692243BE
:101760004C6A22438C6A22431A430260CA68426070
:101770000A6882604968C16030BD00210160416033
:101780008160C160016141618161C1610162416249
:101790008162704710B5114C8CB000212046FFF7D4
:1017A00035FF2046FFF73EFF0D4800900D48002111
:1017B000CDE901016420CDE903018020CDE90501D7
:1017C0000791089109910A9169462046FFF7B8FFF1
:1017D00001212046FFF71AFF0CB010BD580002404F
:1017E000043801408407002010B501218CB0084660
:1017F00002F078FB1E4C00212046FFF707FF204631
:10180000FFF710FF1B4800901B480190002110209B
:10181000CDE902018020CDE90410069107910891DD
:1018200009910A9169462046FFF78AFF01220221A9
:101830002046FFF77DFF01218DF82F1004208DF841
:101840002D008DF82E100E208DF82C000BA802F024
:1018500035F80F208DF82C000BA802F02FF801218D
:101860002046FFF7D3FEFFF795FF0CB010BD000038
:1018700044000240043801402007002030B540F603
:10188000AA21204AC184838B1488E31A9BB20F2BB0
:1018900010D312888283037E002253B11A4BB3F90E
:1018A0000A30062B05DB194B1B78022B03D0002BCB
:1018B00000D1828430BD164B40F68B255B6CA3F2C1
:1018C0002D14AC420FD2428B521C92B24283642A36
:1018D000F0D364224283B0F924208A4201DA02EB79
:1018E0002111818430BD41F29414A342FADBB0F996
:1018F0002430002B02DDA3EB211100E000218184C4
:10190000428330BDF806002060000020EF06002072
:101910003C01002010B50446B0F9020043F69911CD
:1019200048438113E06840F26662504301EBA03007
:10193000E060B4F9001043F6991251438A1321690B
:1019400040F26663594302EBA131216104F020FDAE
:101950006061A18840F6AB2208444010A0F5154113
:101960005539E062914205D9A0F5F851FF39521C72
:1019700091421DD249F25451884202DDA0F5204027
:1019800002E0A0F5F850FF38206300EB400040F380
:101990004F002085B4F924104A42904201DA1046E3
:1019A00002E0884200DD0846E083228461848AE008
:1019B000A0F5FE42FF3A41F255518A4214D8A2F6F0
:1019C000AA20206300EB400040F34F002085B4F9CB
:1019D00024205142E183884201DA084602E0904225
:1019E00000DD1046404250E0A0F5D442AA3A8A42B7
:1019F00015D2A2F6AA20206300EB400040F34F016D
:101A00002185B4F924004242E2832084914201DA24
:101A1000104602E0814200DC0846608453E0A0F5F5
:101A2000AA42543A41F256539A4215D2A2F6AB203A
:101A3000206300EB400040F34F002085B4F92410F0
:101A40004A42904201DA104602E0884200DD084630
:101A50004042E083218419E0A0F5804241F25453D2
:101A60009A4215D2A2F6AA20206300EB400040F370
:101A70004F012185B4F92400E0834242914201DA0A
:101A8000104602E0814200DC0846208462841AE0AD
:101A9000A0F52852AB3A8A4215D2A2F6AA202063BA
:101AA00000EB400040F34F012185B4F92400E083AE
:101AB00042422284914201DA104602E0814200DC77
:101AC00008464042A9E7B4F91E006FF4BF714843CD
:101AD0008013E080B4F92000484380132081B4F9DA
:101AE000220048438013608110BD70471548164A94
:101AF0004FF480410078042821D002F13C03D08AC1
:101B00009B88C01A00B22F2801DD001108E00028D0
:101B100001DD002007E00D4B984201DA184602E093
:101B2000402800DD40209389184400B2884203DC3D
:101B300040F26661884200DA0846908170479181E0
:101B400070470000EF060020B4040020C0FEFFFF35
:101B500038B54B484B4902880B889A1A92B20F2A23
:101B600071D30988484C01804FF0FF01E2884FF49F
:101B70007A7355044FF4967002D51622009103E053
:101B8000950403D515220091014670E0D50402D5D5
:101B900014220091F8E7150502D513220091F3E70E
:101BA000550502D512220091EEE7950502D51122C6
:101BB0000091E9E7D50502D510220091E4E715066A
:101BC00002D50F220091DFE7550602D50E220091C3
:101BD000DAE7950602D50D220091D5E7D50602D5A4
:101BE0000C220091D0E7150702D50B220091CBE71C
:101BF000550702D50A220091C6E7950702D50922AA
:101C00000091C1E7D20702D008220091BCE72289E7
:101C1000550702D507220091B6E7950702D506229F
:101C20000091B1E7D20702D005220091ACE7A27A79
:101C3000D20702D004220091A6E7A289D40603D5D8
:101C400003220091A0E719E0140702D502220091B7
:101C50009AE7540703D4940701D4D20702D0012293
:101C6000009191E70020034602460146009002F0F1
:101C700067FEBDE838400248FFF71AB938BD0000DA
:101C8000040A0020F8060020100A0020F0B5594888
:101C9000594982880B889A1A92B29C2A64D309887F
:101CA000818056490A880146002A0B7843F00201D8
:101CB00056D11646524A1C0715680246127822F081
:101CC000020274D54F4C0746E4887F785FEA845C53
:101CD00002D547F0010701E027F001074770A7048C
:101CE000477802D547F0020701E027F00207477066
:101CF000670401D4E70703D0477847F00807477027
:101D0000640603D5447844F0040404E01C0603D4BC
:101D1000447824F004044470EC0450D4354C9A0701
:101D2000247824F0100423D4324D42782F7A2D7871
:101D3000012A45F0100514D0022A16D02D4C042A91
:101D4000A47804F1010C0CF0FF0C13D0072A25D065
:101D5000032A23D0052A21D0062A1FD021F0100102
:101D600042E0B90702E00570F0BD39070029FADB4F
:101D70000470F0BDFA0601D41A060AD50170022CCF
:101D800004D280F802C0BCF1020FF2D341F080010E
:101D90002AE021F0100101708670F0BD877A7F067D
:101DA000F7D5032C04D8017080F802C0F0BD0FE015
:101DB0005107D8D51906D6D443F0800114E002703B
:101DC0004178CB0701D18907F0D522F010010BE053
:101DD000E9040BD49907E9D4818AC82902D2491CA5
:101DE0008182E3E743F00A010170DFE70270868237
:101DF000DCE70000D0060020F8060020FA060020EC
:101E000098020020100A0020094944F64800088082
:101E1000091D46F648000880091D41F6CC4008809F
:101E20000348001F018841F0200101807047000035
:101E3000182C0140084946F668000880091D0880F2
:101E4000091D41F2555008800348001F018841F0E8
:101E50002001018070470000182C014010B5C28895
:101E600000210AB1032206E002890AB1022202E03F
:101E7000428912B10122027000E0017004784FF42F
:101E8000804344F6206244B1012C06D0022C07D0D6
:101E9000032C01D14180818010BD4380828010BD20
:101EA00041F23331418040F6B731F4E730B5B1F853
:101EB0006A5000231A240D22854202DCB1F9680021
:101EC00030BD4D88854202DBB1F9000030BD01EB29
:101ED00082056D88854201DD144601E013DA134660
:101EE00004EB03024FEA52029A42F0D101EB830263
:101EF00031F8231054889288521A001B424301EB98
:101F0000622000B230BD31F9220030BD054920B158
:101F1000086940F080000861704703484860034842
:101F2000486070470020024023016745AB89EFCD30
:101F300006494FF47A70CA68D20705D0401E0004E3
:101F4000000CF8D1FF2070470020704700200240AD
:101F500011480321A0F14C0280F836100021518174
:101F60000E4A1186D162D1831184518481620C4959
:101F70008A6CB2F5206F01DBA3228262897A11B1EB
:101F8000816A49428162C16A41F391018162880399
:101F90000449486270470000600000201C050020D2
:101FA0003C01002064080020044900204881088189
:101FB000C8628862024948627047000060000020E1
:101FC0008C080020F0B53B4988894A89801A80B284
:101FD0000F2866D388894881CA8937480B3A272A4F
:101FE00026D28A7822BB8268364B42F480728260A5
:101FF000324A354C354D12785607314A0AD4344EA0
:1020000036881680334A12881A80334A1288228012
:10201000324A09E0324E36881680324A12881A80D7
:10202000314A12882280314A12882A8001228A701D
:102030002F4B304D19469A7F0968802A32D302F01F
:102040001F0255F8222011422CD0826822F48012FF
:10205000184E8260123614461215B778521C62F37D
:102060008617254AB77093F816C01778BCF1800F11
:1020700027F0020608D30CF01F0C55F82CC011EA0B
:102080000C0F01D147F0020616701A7E802A0DD37C
:1020900002F01F0255F82220114207D144F400211A
:1020A0008160F0BD826842F48012D1E724F40021FF
:1020B000F6E70000EC060020980200203C0100201A
:1020C000AC040020AE040020B0040020B2040020C4
:1020D0009C0400209E040020A0040020A2040020F4
:1020E000A4040020A6040020A8040020AA040020C4
:1020F000CC0500202C910008B404002070B52048C5
:1021000081890289891A89B20F292FD38189018196
:102110001C4B1D4819465D7A06681C4C096846F040
:102120000402802D07D305F01F0554F825502942DD
:1021300001D126F0040202609A7B802A17D302F0B4
:102140001F0254F82220114211D1026822F002022B
:102150000260DA7A802A0ED302F01F0254F822209D
:10216000114208D1016821F00801016070BD0268C8
:1021700042F00202ECE7016841F00801F5E70000D7
:10218000EC060020CC050020980200202C910008CD
:10219000F0B51D4C1B4A4FF0010C94F83B5094F8DD
:1021A0000AE0144692F83C3094F838402B43651C02
:1021B000EEB2154D95F83D700025BEF1FF0F0AD027
:1021C000BEF1000F06D18B4213D155700C2C01D2F9
:1021D00082F83860F0BD834202D182F801C0F5E791
:1021E0008B42F7D15570B80709E000BF82F838502C
:1021F000F0BD8342FCD1F84382F801C0800700287B
:10220000F4D0F0BD3C0400203C010020F0B5CA78B9
:10221000002502F00F03D20601D58A7813430A780D
:102220004FF00F0E12F0FF0F4FF001021CD00468A8
:102230000F8802FA05F63740B74211D14FEA850CF4
:102240000EFA0CF724EA070703FA0CF43C43CF78A4
:10225000282F02D0482F02D002E0466100E006613C
:102260006D1C082DE4D304600C88FF2C1ED9446833
:102270005FF0000606F1080702FA07F50F882F4005
:10228000AF420FD14FEA860C0EFA0CF7BC4303FAAB
:102290000CF73C43CF78282F00D14561CF78482FE9
:1022A00000D10561761C082EE4D34460F0BD000027
:1022B000F0B5144C002801DAE36900E06368420DD0
:1022C000120185B2C0F301579540C0F30346032FB6
:1022D00005D0C2020AD50322B240934307E023F09F
:1022E0007062636823F07063636002E0AB4343F0A5
:1022F000706201B12A43002801DAE261F0BD626038
:10230000F0BD0000000001400246002092680A4231
:1023100000D00120704741617047016170470AB1E8
:1023200001617047416170470F4A104B92F83810B5
:102330005B5C834201D1012004E00D4B5B5C834276
:1023400003D1002082F83A0070470A4B5B5C83425D
:1023500001D18120F6E7084B595C814201D18020F0
:10236000F0E70320EEE700003C010020EC940008B9
:10237000FE940008F2940008049500080A4810B57D
:1023800001784FF000024C0708494FF0FF038968BD
:102390004FEA017105D5002901DA827210BD8372FE
:1023A00010BD0029FBDBF8E73C010020980200206B
:1023B000F0B5194E194C0022E31CA6F1060CB75CCF
:1023C000A518ED78FF5C0D430F43BD421FD01CF8EC
:1023D0000270FF5C0F43BD4219D015460023A618BA
:1023E000F6780E43C6545B1C1CF80220DBB2062BA9
:1023F000F5D3C17881700179C17000214218491C60
:1024000015711CF80550C9B20629F7D3F0BD521C4E
:10241000D2B2032AD3D3F0BDBE8C00083C04002006
:1024200010B502460021064B06205C1864789442E1
:1024300000D10846491CC9B20629F6D310BD0000D8
:102440003C010020214810B590F867100022204878
:10245000012936D11F49898899BB1F491E4B4C6CF5
:1024600040F6B831B3F86E308C4227DD1B4909784D
:1024700021BB90F82711491CC9B280F82711C8293F
:102480001CD380F827210146D0F82C4191F828115F
:10249000A34203DD052908D2491C01E041B1491ED0
:1024A00080F82811C9B2052902D3012180F826112C
:1024B000191B074C2C3C6162C0F82C31B3F5FA6F44
:1024C00003D280F8262180F8282110BD680C002056
:1024D00098020020C60500203C010020EF060020E5
:1024E0004FF4C0428260002141620E22828141F29B
:1024F00062020261082282824FF46042C28201833A
:102500004FF07842C0E9072140F6C41101807047BE
:10251000B0F90010B0F90220891A41600269037D08
:102520004A431A41436A13444362026A934200DDFC
:102530004262436AC269934200DA42628268436A35
:102540004A43017B0A410B41D118B0F918208A4255
:1025500001DA10467047B0F916008842FADC08B27A
:102560007047000010B514481449B0F88C200B884F
:102570009A1A92B2B2F5437F1DD90988A0F88C103F
:10258000B0F88A1020F8581F002242860C480D4CE3
:10259000C2888280C180C38983812489891AA4B2B8
:1025A000C4818160E11A0161074A818AC182928AED
:1025B0008282511A816110BD3C010020F806002082
:1025C000300C00201C0500206000002009480A494A
:1025D000B0F8AA200B889A1A92B241F684639A4204
:1025E00006D3098820F8AA1F4188818000214180F4
:1025F000704700003C010020F80600200D480178DB
:10260000C90702D00C49098801E04FF6FA71C1658B
:10261000094901201039088007482438018841F011
:102620000101018004481838018821F01801018057
:10263000704700003C010020240400400A49D1F802
:10264000902012B1521EC1F8902031F88A2F521CEE
:1026500021F81A294A6A521C4A628A8F521C8A87B8
:1026600001F8380C704700003C0100201CB52D48D3
:1026700090F83B3090F83C20934252D000248DF8E3
:10268000044053408DF800309DF800300122012BAA
:1026900008D09DF80030022B09D09DF80030042BA3
:1026A0000AD00DE01F498DF80420443108E01D498F
:1026B0008DF80420463103E01A498DF80420483192
:1026C0009DF80420012A2CD190F83D309DF800405F
:1026D000154AA34217D090F83E309DF8004023429F
:1026E00008D0B0F84C30A0F84A300B881488E31AB0
:1026F000A0F84C3090F838302BB1B0F84030148846
:10270000E31AA0F8423012880A80A0F8402010F89E
:102710003E1F9DF80020114300F801199DF800109C
:1027200001701CBD3C040020F806002070B5344D3B
:1027300040212846FFF7E8FD840080212846FFF766
:10274000E3FD44EA4004A9152846FFF7DDFD0443F4
:10275000E1B22C4C94F870508D4250D04D4084F82A
:102760007010012D03D0022D01D0042D47D194F813
:102770007400A84384F8740094F87320AA420FD020
:1027800084F8735094F8722001238B401A4207D1C9
:102790001A4384F8722094F87110491C84F871105F
:1027A00094F87110042928D330B1012811D00228DF
:1027B0000FD004280DD012E01348C18821F0400149
:1027C000C1802078002184F83B1020F06000207048
:1027D00005E0217841F02001217084F83B000B498D
:1027E00094F83B0091F82720904204D081F827000C
:1027F00007492020087000F00DF884F84C5070BD97
:10280000001001403C010020100A0020680C00204C
:10281000EC06002070B50D4D40212846FFF774FDF1
:10282000840080212846FFF76FFD44EA4004A91583
:102830002846FFF769FD04430548072100F8704F5B
:102840000171002141708170C17070BD00100140A4
:102850003C01002070B5344890F83A10CA43920702
:1028600061D001F0030280F8392090F83D305B061A
:102870001B0E80F83D30012A01D0812A02D15B1C59
:1028800080F83D300278D2074DD0DBB203F0010270
:10289000C3F34004A24246D1B0F84E400025641C68
:1028A000A0F84E40204CA0F8505090F83E60A47A1A
:1028B000B24202D080F83E200DE0A607B6EB837F3F
:1028C00002D080F83F5006E090F83F30642B02D2EF
:1028D0005B1C80F83F3090F84030642B0CD25B1CBE
:1028E000DBB280F84030022B06D204F001039342A1
:1028F00002D1022280F84020012901D0002912D102
:1029000090F83820C16D00EB820291610163D0E93B
:1029100006121144D0E908231A441144826A114472
:10292000C26A1144416370BD3C010020FEE7000013
:102930002DE9F04F00BF00209E4E9F4AA6F5127170
:10294000A6F5BE79A6F1440B06F1440E804601F5CA
:10295000E074A1F1780301F5457A1D5C15F0C0071C
:1029600006D0402F51D0C02F77D0802F76D004E1F1
:1029700015F01F0504D0154440F080072F7201E0C8
:1029800082F80880012826D0022824D0032822D0EB
:10299000042820D008281ED010281CD0874D55F8B8
:1029A00020C0DCF8005054F820703D40CCF80050B6
:1029B000824D55F820C0DCF8005056F820703D4399
:1029C000CCF800501D5CAD0659F820502F6813D587
:1029D0003AF810C03EE051F820502F6854F820C05B
:1029E00007EA0C072F6051F820502F6856F820C0D6
:1029F00047EA0C072F60E5E7DFF8B8C10CF1F00CEF
:102A00005CF820C007EA0C077EE015F01F0504D033
:102A1000154440F080072F7201E082F808800128F9
:102A20001DD002281BD0032819D0042817D008284D
:102A300015D0102813D0614D55F820502F6854F848
:102A400020C007EA0C072F605C4D55F820502F6816
:102A50005BF820C047EA0C0756E00BE056E051F85F
:102A600020502F6854F820C007EA0C072F6051F857
:102A70002050ECE715F01F0505D0154440F0800705
:102A800085F8217001E082F82180012825D00228F4
:102A900023D0032821D004281FD008281DD01028B7
:102AA0001BD0464D55F820C0DCF8005054F820707B
:102AB0003D40CCF80050414D55F820C0DCF80050A6
:102AC0005EF820703D43CCF800501D5CAD0615D576
:102AD0003A4D3AF81070CC3514E051F820502F6878
:102AE00054F820C007EA0C072F6051F820502F68D7
:102AF0005EF820C047EA0C072F60E6E72D4D3AF854
:102B00001070E03D55F820502F6036E015F01F059D
:102B100005D0154440F0800785F8217001E082F867
:102B20002180012830D002282ED003282CD0042860
:102B30002AD0082828D0102826D0204D55F820C0AB
:102B4000DCF8005054F820703D40CCF800501B4D8C
:102B500055F820C0DCF80050164F883757F8207021
:102B60003D43CCF800501D5CAD06B1D4114F3AF88E
:102B70001050E03F57F820703D60401CC0B2112853
:102B8000FFF4EBAEBDE8F08F51F820502F6854F8F9
:102B900020C007EA0C072F6051F820502F68DFF89B
:102BA00014C00CF1880C5CF820C047EA0C072F60B9
:102BB000D9E70000B8930008CC050020B4910008C4
:102BC0004FF40771C1824FF45861018340F61451EC
:102BD00081837047F0B5C48AB0F900608681B0F98E
:102BE0000250C581B0F9043002270021012203827E
:102BF000AB4204DBB54202DDC78042810CE0B34248
:102C000004DBAE4202DDC78041811CE09D4205DB52
:102C1000B34203DDC2804781018115E0B54204DB88
:102C20009E4202DDC280418105E0AE4205DB9D424D
:102C300003DDC1804281078106E09E4204DBAB4296
:102C400002DDC18047810281C388458900EB4307CB
:102C500000EB4505BB89AE899B1B0FFA83FEA0F8EC
:102C600012E00689AB8900EB460CBCF80CC0A3EB64
:102C70000C038382B0F91830B7F90CC0A3EB0C0C2D
:102C8000B4EB4C0F04DA80F82010A3F1A10113E09B
:102C9000A64503DD80F82010B9890BE026B1012E8E
:102CA00004D0022E10D004E0062100E0052180F8B7
:102CB0002010A989091B6D31418309B2B1F5586F04
:102CC00004DB5B1E438304E00421F0E7002900DC01
:102CD0004283418B8183F0BD0B49002288760A62D2
:102CE000CA614A62094A32F9103002EB40028B6233
:102CF000B2F90220CA62064A32F810000882A1F82E
:102D00006000A1F862007047EC01002016950008F1
:102D10000A9500082DE9F05FFC48FD4982880B8880
:102D20009A1A92B20F2A44D3098882468180F948C0
:102D30000127F94C0188F94E002579B3491E01801D
:102D4000E573F74AA5622068B2F90220430742F60C
:102D5000AA2118D4F38843F40053F380F04B1B7876
:102D60009B0709D5A36823F08003A360A4F87C50D7
:102D700084F87E5084F87F50C30404D484F8F07043
:102D8000C4F8EC5003E084F8F050430707D48A42BB
:102D900005DB84F8F470A4F8F25004E010E084F845
:102DA000F450430703D48A4201DBC00703D084F800
:102DB0001151BDE8F09F84F81171A4F81251F8E7A1
:102DC000B4F8180143F69821884202D2401CA4F8B6
:102DD000180101F0CBFDDFF84C83DFF830B398F831
:102DE0005000ABF1180B10B1FEF76CF905E09BF841
:102DF000001021F001018BF80010FFF723FB00F019
:102E0000D7F9C94841F26801436C4FF400608B4226
:102E100001DBC64904E0B3F57A6F02DAC349091D44
:102E2000086098F85100C646C107DFF8EC82C04838
:102E3000DFF80093A8F12C0838D0817B802931D3AA
:102E4000217889072ED4E27B88F80520B44A4146D0
:102E500092F800C02CF0020C82F800C0ABF80250CF
:102E6000CBF814509BF800C02CF0010C8BF800C07C
:102E7000B279520611D44A89B2F5FA7F03D2521CB4
:102E8000A8F80A2012E040F63C70834201DD0020E1
:102E900011E1082088F803700DE1CD700020A8F83A
:102EA0000A5008E188F80350A8F80A50A1680A05FA
:102EB00001D50820FFE0F4469EF83FE05FEACE72BD
:102EC00041D0E27B88F80520437A802B45D32378D4
:102ED0005B0731D4F3889B0404D500BF21F02000A8
:102EE000A06030E0ABF80250CBF814509BF800C063
:102EF00041F020012CF0010C8BF800C0A160C17DD5
:102F0000802909D301F07F0300684FF00041D940C8
:102F1000084201D1277100E025712079C00702D154
:102F20005FEA8E7005D50320032A01D088F8087067
:102F3000C1E00020A562BEE021F02000A060F08882
:102F400020F40050F08094F8260101280AD09CF863
:102F5000630048B1FDF776FF0FE0206840F0040001
:102F60002060BBE70920A6E0A068C10502D520F0DB
:102F7000080001E040F00800A06094F8467043F2B9
:102F80001E5343F23331BFB143F69912012F23D0C0
:102F900099F80010684B43F6FE70032FC1F38101CE
:102FA00028D001293DD002293BD093F8561004299E
:102FB00034D0A4F814013AE099F80000C0F381007D
:102FC000012806D0022804D0A4F81431A4F8441033
:102FD00032E0A4F81411F9E799F80000C0F3810079
:102FE000012804D0022802D0A4F8143122E0A4F869
:102FF00014111FE001290AD0022908D093F85610B5
:1030000004290BD0A4F81401A4F8440014E0A4F897
:10301000140193F8561004290CD0F5E7A4F81421F4
:1030200008E0A4F8140193F85600042802D04FF4E5
:103030008040E9E7A4F84420FEF744F89BF800102C
:10304000C90702D0BBF8021001E035488188AAF810
:10305000121008B2B4F944104FF480424843C0F350
:103060008F314046A8F81210914200D9428233496C
:103070000978C90605D5428A41F233318A4200D225
:1030800041822189C1F3C002C1F300218A4205D1E6
:10309000428A40F6CC418A4200D94182B17AC907BE
:1030A00000D04582B8F81200A06200287FF7EFAE8A
:1030B0002348057002209AF81A1099B9022841D0C5
:1030C00080B119490B789D0608D5B5796D0605D5EF
:1030D0001A4D2D78ED0965F386130B70F18821F4F4
:1030E0000A61F1801049496C4E290ADBF1880B0610
:1030F00007D521F08001F18009490B7823F0020304
:103100000B708AF81A00E07353E6000020090020D3
:10311000F8060020FA06002098020020100A00207D
:10312000C6050020680C00203C010020100C014066
:10313000CC050020B404002060000020D006002050
:103140000C070020B9F83830002BBAD143F6982389
:10315000A9F83830B5E770B500230C8863F30F0287
:10316000012505FA03F6344206D0C3F10F0605FA2D
:1031700006F1114361F30F025B1C102BF1DB02809F
:1031800070BD70B500230C7863F30702012505FAC2
:1031900003F6344206D0C3F1070605FA06F11143DF
:1031A00061F307025B1C082BF1DB027070BD0000AD
:1031B000F0B51F4890F866301E48012B816821F455
:1031C000006232D11C4BDE8874062ED41B4D0F05D5
:1031D0004FF00004B5F902501ED4194A526C642A0B
:1031E00011DC40F6386295420DDAB2040BD4027855
:1031F00052070ED4B0F8D42040F6B835AA4203D214
:10320000521CA0F8D420F0BD41F4006181605C81C3
:10321000F0BDA0F8D440F0BD41F2CD018D42FADD01
:10322000997AC907F7D18260F3E78260F0BD0000A8
:10323000680C002098020020100A0020C60500201B
:103240003C010020F0B5364D364F044695F83B0062
:1032500097F83B1023780843EE1C6278834205D12F
:10326000E0781146FEF794FF207908E094F802C058
:1032700084450CD1E1781046FEF78AFFE07905F825
:103280002F0F2878805D6870287BE877F0BD824238
:103290001DD161461846FEF77BFF95F84E1095F854
:1032A0003B00814207D1B97A09B1A17900E0617987
:1032B00085F82F101EE06978012901D0A17922E05C
:1032C000617927E0297841F00401297012E0E17862
:1032D0008142DBD119466046FEF75AFF95F84E1041
:1032E00095F83B0081420AD1B97A09B1617ADFE7EA
:1032F000217ADDE715F82F1F895D6970C5E76978C8
:10330000012906D0617A85F82F10B97A0029F1D108
:10331000D8E7217A85F82F10B97A0029EAD0D1E7C9
:103320003C0400203C0100200B48017821F0020100
:1033300000F8381B002100F81819417781773321F4
:103340008185418508214184012100F81F1C034823
:1033500080F83910704700003C0400203C01002038
:103360000D4900B50B4851F8012F40F8032F89880B
:103370008180084801210930FFF71AF80548022129
:103380001330FFF715F8034804211D305DF804EBF6
:10339000FFF70EB83C0400203C010020094944F628
:1033A00048000880091D46F648000880091D41F2C2
:1033B000111008800348001F018841F0200101809E
:1033C00070470000182C01402DE9F047664C674B10
:1033D0000025A0780126654A103305287ED2DFE853
:1033E00000F00313113E1100108820F0010010803E
:1033F0001D805F480580001F0580001F0580FFF7C6
:10340000CDFFA670BDE8F087594941F244401C3910
:103410000880574945F6580024390880091D47F2AD
:103420005800088052492020283908800020401C7C
:10343000C0B27328FBD3FFF7B1FF4C4984F85C504E
:103440002C3147F6906008804848143006801D8073
:10345000108840F0010010800220A070D2E7002107
:103460005FF0010004EB410204EB4003B2F850208E
:10347000B3F850309A4200D20146401CC0B2062830
:10348000F0D33C48405C84F83900FFF74DFF1D2025
:1034900000F0F3F900F076F8374E38484FF48079B1
:1034A00096F83B10012904D002291BD0042930D002
:1034B00047E040218046FEF727FF870080214046F5
:1034C000FEF722FF47EA400749464046FEF71CFF49
:1034D000074347F0010084F83B0000E03DE022484C
:1034E00009302CE040218046FEF70EFF8700802146
:1034F0004046FEF709FF47EA400749464046FEF7C7
:1035000003FF074347F0020084F83B0016481330DE
:1035100015E040218046FEF7F7FE870080214046F7
:10352000FEF7F2FE47EA400749464046FEF7ECFE4A
:10353000074347F0040084F83B000B481D3002F0BD
:1035400001FE94F82F0086F838001D2000F0ABF93A
:103550000420A0700A48057054E7108820F001008C
:1035600010801D80A5704DE73C040020000800403D
:103570003C2C0140C48C00083C010020001001409C
:10358000EF0600202DE9F041344C14F82F0F344D94
:10359000E07240212846FEF7B7FE860080212846CB
:1035A000FEF7B2FE46EA4006AF1539462846FEF75A
:1035B000ABFE0643207BF1B22F3C814215D084F84C
:1035C0003C0040212846FEF79FFE860080212846C9
:1035D000FEF79AFE46EA400639462846FEF794FE74
:1035E000064384F83B60FFF741F81E4D95F83B0019
:1035F000012827D0022828D0042829D0174894F879
:103600003B102730085C04F8300F14F80109FEF76E
:1036100007FF04F82F09A87A00B10120607001F0BB
:103620003DFA94F84E0094F83B10884206D094F886
:103630003800062802D2401C84F8380084F84E1066
:10364000BDE8F0810548093004E00448133001E08A
:1036500002481D30BDE8F041FFF7F4BD3C040020F6
:10366000001001403C0100202DE9F041524991F841
:103670007200AA287ED191F8730055287AD14F4C58
:1036800000200A5C2254401CC0B27428F9D34C4E6E
:103690002069C6F80100A08AA6F80500D4F8160033
:1036A000F060D4F81A003061D4F81E001234706152
:1036B00002F0EEFC4349608A888102F003FD207D20
:1036C000123CC007307802D040F0040001E020F046
:1036D00004003D4930704FF480403C4D886114F83F
:1036E000280F85F82000608B6880A08BA880E08B75
:1036F000E880208C2881608C354F688194F8240004
:1037000087F8D20014F8011C304686F83B100026DA
:10371000C0F89460FFF724FE2E48A18E0183E18E4D
:103720004183218F818394F84210283C012908D0DD
:10373000022901D0032909D0297821F00C01083190
:1037400007E0297821F00C01091D02E0297841F0F9
:103750000C01297094F86E20012162B1012A01D078
:10376000022A0BD087F8461094F864301A4A4BB1FD
:10377000518108E014E087F84660F5E7022287F8F7
:103780004620F1E7568194F8701001290AD094F888
:103790006D1051B101290BD04FF48051A0F8761073
:1037A000BDE8F08144F21C71F8E74FF40051F5E7F1
:1037B00041F25551F2E7000000FC0008680C0020BF
:1037C0003C01002060000020000C0020B404002018
:1037D000980200201C050020100A00207CB5012161
:1037E000082000F0A3FB4FF48070ADF80400102413
:1037F0008DF8074001208DF8060001A91548FEF755
:1038000005FD0121092000F091FB01211248FEF77E
:103810004FFD0820ADF8000004208DF803000F4E86
:1038200003258DF8025069463046FEF7EFFC08216B
:103830003046FEF770FDADF800408DF803408DF87E
:10384000025069463046FEF7E1FC10213046FEF793
:1038500062FD7CBD0014014000023000000C0140FC
:10386000FEE7704700F01F020121914040098000EF
:1038700000F1E020C0F88011704700F01F02012124
:1038800091404009800000F1E020C0F880117047AD
:1038900000F01F02012191404009800000F1E0206A
:1038A000C0F80011704700F01F020121914040094B
:1038B000800000F1E020C0F80011704770B50F23C0
:1038C000C47801780122F4B1144C2468457804F4DA
:1038D000E064C4F5E064240AC4F10406E34084789B
:1038E000B5401C402C4301F1E021230181F8003454
:1038F000007800F01F018A404009800000F1E020BC
:10390000C0F8002170BD01F01F008240480980000E
:1039100000F1E020C0F8802170BD00000CED00E057
:103920000249084302490860704700000000FA0598
:103930000CED00E02DE9F05F00261D20FFF792FF5F
:103940006C4CDFF8B4B1A4F1B000A77E90F8381049
:10395000DFF8A8E1DFF8A8A100258F427ED0E77646
:10396000A176626A036B5A434FEA12499BF808201A
:10397000120702D51EF8012000E00A4694F812C092
:10398000BCF1010F09D004EB4206B6F902C0C4F83D
:1039900028C0B6F90460E6620CE043F6FF7CC4E997
:1039A0000A5C90F83DC05FEACC7C01D012B102E025
:1039B000052A00D1012600EB47074FF0804CBF8954
:1039C0003F04B7FBF3F3E361476BBCFBF7F72762F8
:1039D00094F813C0BCF1000F06D0BCF1010F05D064
:1039E0003B4403EBD3735B10636201E03B466762C9
:1039F000DFF810C14FF6FF7707EA8307ACF80870CD
:103A00009AF8007090F80A8090F83DC0082F08F0EE
:103A100003070CF0030C05D067450BD1B8F1000F7C
:103A200005D008E0674505D0B8F1000F03D05B4230
:103A3000636200E06562C6B1636A002B03D006DDF5
:103A4000228D05E00AE0304B33F8122000E0A28D11
:103A5000A4F86020227822F0200222709AF8002038
:103A6000042A07D0082A05D012E0B4F8603003EB2E
:103A70000902EDE780F8405065629BF808000007F6
:103A800001D51EF80110204830F81100A4F860009C
:103A90001E49606A09883E314843B4F8601001EB62
:103AA000204006B21D20FFF7F3FE606A002807D011
:103AB00021784FEA81600ADD002804DAA08D09E050
:103AC000B4F8600006E0E06AB04208DB0CE00028D1
:103AD00002DA208D208208E0A06AB04204DD208254
:103AE00041F02000207000E026822575657525864E
:103AF000BDE8F09FEC01002098020020F894000837
:103B0000EF060020E80900200A9500082404004080
:103B100043184FF48042934210DD904202DD10467C
:103B200000210BE0914202DD0020114606E08003F7
:103B3000B0FBF3F000B2C0F5804109B241EA0040A9
:103B40007047F0B5002240F2AE440E258460426218
:103B5000858144F24C2608270661878243F6FF7C64
:103B6000C282A0F818C040F249234FEA8C3E43605D
:103B7000C0E9072E8C604A628D810E618F82CA82F5
:103B8000A1F818C04B60C1E9072EF0BD00214162C9
:103B9000094981600E2181814FF6BF5101610821E1
:103BA00081824FF44041C18243F6FF7101830907CE
:103BB000C161024901627047638A010000C0FF0FC2
:103BC000064941F6A260088005480168054A01F4EB
:103BD000E06111430160BFF34F8FFEE7442C0140C9
:103BE0000CED00E00400FA0538B501210D2000F0CD
:103BF0009DF94FF4E060ADF8000018248DF8034003
:103C000003258DF8025069460D48FEF7FFFA4FF480
:103C10006040ADF800008DF803400A4C8DF802506A
:103C200069462046FEF7F2FAA014ADF800004820DD
:103C30008DF8030069462046FEF7E8FA38BD00001B
:103C400000080140000C0140F0B50121CE028DB00A
:103C5000304600F06BF9594F384601F091FB08A847
:103C600001F0BAFD4FF45860ADF824000024ADF81F
:103C700020402020ADF82200ADF8264008A93846A3
:103C800001F05CFD0021384601F0AFFD4FF6FF71F9
:103C9000384601F0B4FD01220021384601F040FD14
:103CA0000121384601F028FB04A801F040FBADF8E3
:103CB00010607010ADF81200ADF81440A220ADF8FD
:103CC00016007000ADF81800ADF81A40ADF81C40B1
:103CD00004A9384601F01AFB6025ADF80050ADF894
:103CE0000440ADF80840ADF80C40ADF80240ADF826
:103CF0000640ADF80A40ADF80E406946384601F07E
:103D0000FFFB6946384601F041FC6946384601F040
:103D100087FCADF800500125ADF8045040F6145072
:103D2000ADF80600ADF80840ADF80C40ADF8025013
:103D3000ADF80A40ADF80E406946384601F0B4FCD3
:103D40000121384601F0FCFA0821384601F018FC40
:103D50003146384601F05AFC0821384601F09EFCF5
:103D60003146384601F0D2FC7021384601F0DBFCC8
:103D700018208DF82C008DF82D408DF82E408DF8F0
:103D80002F500BA8FFF79AFD0C480C30018841F02A
:103D90008001018009481430018841F0010101804F
:103DA000001F04800121384601F0D4FA8DF8285014
:103DB0000121384601F0D8FA0DB0F0BD002C0140C9
:103DC0007047000070B50189C1EB411101EB410161
:103DD000CA0B42810B49104603F010FD09480C380C
:103DE000B0F90C200168B0F90E4001FB02F5436800
:103DF000614303FB145503FB0211AD138913C0E9A2
:103E0000055170BDF409002040F2134141600821C2
:103E100081608621C1604FF4804101614942416166
:103E200000210162C16270470162704710B50188CC
:103E30004288891A09B20183B1F5005F02DBA1F55E
:103E4000804104E011F5005F02DC01F5804101834F
:103E5000B0F9182041685143C1618368846A5343B3
:103E6000C2681B12624303EB2222036A1A44114404
:103E700002628A13426241698A4203DB01698A4213
:103E800000DC11468A1AC0E90A21028E4FF403733E
:103E9000594302EBA13202860B4A1278082A04D158
:103EA0000A4A136F03EBA1311167B0F93010B1F575
:103EB000804F02DDA1F5804103E0002902DA01F51F
:103EC0008041018610BD0000EF060020240A00207A
:103ED000034A516821F4404101435160704700009A
:103EE00000100240044A0029516901D0014300E05A
:103EF000814351617047000000100240044A0029CC
:103F0000D16901D0014300E08143D16170470000D5
:103F100000100240044A0029116901D0014300E069
:103F2000814311617047000000100240044A0029DB
:103F3000916901D0014300E0814391617047000025
:103F400000100240044A0029D16801D0014300E07A
:103F50008143D160704700000010024030B5244911
:103F60004A6812F00C03234A03D0042B01D0082B1B
:103F700026D002604A680F231F4C03EA1212A35C8A
:103F80000268DA4042604B68072505EA1323E35CC8
:103F900022FA03F383604B6805EAD323E35CDA403B
:103FA000C2604B68032403F4404104EA933303EBFB
:103FB0009161114B1B1F595CB2FBF1F1016130BDE6
:103FC0004A680E4B1A404B68140103F4803303D542
:103FD000C2F38342113202E0022404EB924213B195
:103FE0004B689B0301D5064B00E0024B5A43C0E7E8
:103FF0000010024000127A000400002000003C087B
:1040000000093D002DE9F041274CA615402120462E
:10401000FEF77AF9850080212046FEF775F945EA1A
:10402000400531462046FEF76FF90543EDB24021C9
:104030002046FEF769F9870080212046FEF764F9E3
:1040400047EA400731462046FEF75EF90743F8B2DB
:10405000A842DBD140212046FEF756F98700802197
:104060002046FEF751F947EA400731462046FEF761
:104070004BF90743F8B2A842C8D140212046FEF7C9
:1040800043F9870080212046FEF73EF947EA4007C2
:1040900031462046FEF738F90743F8B2A842B5D1B9
:1040A0002846BDE8F08100000010014010B502680C
:1040B000416802FB02F301FB01330D4CA34211D90D
:1040C0001B0E0E3B0B4C9BB212B234F8133009B2EC
:1040D0005A43594342F38F3241F38F31C0E90221F1
:1040E000012102E0C0E902210021017410BD00009D
:1040F000E10BBF0E208800082DE9F05FFE48FF4964
:1041000002880B889A1A92B20F2A7DD309880180FF
:10411000FB4802468189D2884B0703D48B0701D420
:10412000CB0702D042F4007201E022F40072C28098
:104130008146080702D44846C90604D5B9F80610D6
:1041400041F0010102E0C18821F00101A9F8061047
:10415000EB48FDF783FEEB484FF4804BB0F93A1083
:10416000594502DA491C418702E0E649A1F83AB014
:10417000E54E41F6CC40E54DB16C814203DDA868C7
:1041800020F01000A860E249DFF888830024088846
:1041900028B1401E0880EC7388F8004028E0B9F888
:1041A000060042041BD4B9F80C10CA0617D409073C
:1041B00015D4010613D4810611D401050FD441068C
:1041C00003D5D5490978090609D5410707D4C105A2
:1041D00005D4010703D4810401D4C00608D5CF4813
:1041E000EC73CF4988F80040C4830C8080F82A40E3
:1041F000EA8FCC48CC4942B1521EEA87027822F0BD
:1042000002020270EC730BE08DE0027842F00202D1
:10421000027098F80000012804D10878062801D11E
:1042200088F8004098F80000DFF8E0A20127AAF122
:104230002C0A0A2879D2DFE800F0F1760576F0EF53
:104240007678F6EDE87B09281AD0DFF8E0920228AC
:1042500076D0B5F8400010B399F8680040F63A22DD
:10426000012822D0C5F8D84085F8EA40CAF8204095
:10427000B5F9301001F21D50904226D8102325E0E8
:104280009D484430FEF72CF9FDF762FE716CCAF8C8
:10429000281041F27C510920CAF81810BAE1A4484C
:1042A00041892986A5F8407015E0A248C5F8D800D4
:1042B00085F8EA70B5F9301001F21D53934201D828
:1042C000102300E02023102202E0202310220020EF
:1042D00000F042FB288699F868209749012A726C01
:1042E00040F2DC504FF4927311D0824204DA9048CD
:1042F000B0F90A00984211DBB5F8403040F6C4101E
:104300005B1C9BB2A5F84030834207D20FE082428B
:1043100009DA8748B0F90A00984204DA88F80040C0
:1043200085F8EA404C83BDE8F09F16E108E0754847
:10433000C0680028F7DC45F2F0508242EEDAF2E77E
:10434000706CCAF828008AF807707C4FA5F84040C6
:1043500085F8EA40797F564699B1F87F80B3288D79
:10436000B5F9301000B20A23052200F0F5FA2886CC
:10437000FC777C77B5F93000584550DDA5F830B0B2
:10438000D1E795F8461000B2022916D06C4900BF5B
:1043900001F044FCA5F8E400A96A00B2814200DA09
:1043A000084600B2B08299F84D104F460029B5F981
:1043B000301006D03623052206E06149B031E7E728
:1043C00024E040F24713102200F0C6FA2886B5F91F
:1043D0001601B5F91411884208DA97F84D1011B199
:1043E00000F102000CE000F1080009E00BDD31797A
:1043F00001F10101C9B231710229BBD33471401EF0
:10440000A5F81601B6E7A5F81611B3E740F2666005
:104410002886AFE728E006E04CE047E04FE00028C0
:1044200081DA2C867FE74748D5F8DC10814202D23A
:10443000491CC5F8DC10E97B082903D1D5F8DC104C
:1044400081420DD388F80040A868C10502D520F04C
:10445000080001E040F00800C5F8DC40A86062E711
:10446000BDE8F05F02F02ABCE87B092801D02C8669
:1044700043E1DAF81C005746401CCAF81C00022829
:1044800009DD388D012301B2388B052200B200F01E
:1044900063FAFC61B8621848398D44300180B6F87F
:1044A00044104180FEF734F828863CE7BDE8F05F11
:1044B00004F078B82448007809287DD033E7234BEE
:1044C000DFF88CE01888401C82B222481A80C82A83
:1044D00004D390F800C0BCF1010F4AD0B2F57A7F46
:1044E00004D390F800C0BCF1020F42D0B2F5FA6FCD
:1044F00033D30278032A2FE020090020F806002099
:10450000100A00201C0500203C0100209802002019
:10451000FC060020EF060020D0060020B408002092
:104520001E000020C6050020F0060020680C0020B8
:104530006000002034F3FFFF90090020300C0020C1
:10454000568B0008C0D40100540200201600002041
:1045500014000020150000200BD0E87B801E0828E6
:1045600073D2DFE800F01191CDDE05E9690487E63A
:10457000D9E604701C80B9F8062022F40062A9F87C
:1045800006208EF80070E8E7FDF7F8FE3078400668
:1045900011D56D48807804280DD0706C82280ADA15
:1045A000B07A96F83D1000F0030001F00301884254
:1045B00001D001F033FD00E09FE098F800000628EC
:1045C000D6D086F83F40B06C43F2333148435F4960
:1045D0008013C86281035E484162FDF7B9FC8AF826
:1045E0000770B5F81401A5F81601706CA5F88240A3
:1045F000B0F5437FA5F880B00FDDA86840F4806077
:10460000A86096F838100529B2D100BF40F010001C
:10461000A86070E088F8000085E6A96821F4806150
:10462000A96040F28A21884204DA3078400601D439
:1046300002F030FAA868E9E7706CB0F5437F05DA5C
:104640000878062802D00C706EE075E041480178C9
:1046500021F040010170FDF77BFC43F6FE70A5F8E8
:104660001601DC35FDF78AFE3B4810F82C1F21F0BF
:104670000101017039492C604C6235494C620821B6
:1046800088F8001044644EE699F80600C006C3D4CA
:10469000706CB0F57A7F30DDFDF770FE3078400643
:1046A00011D52948807804280DD0706C82280ADA48
:1046B000B07A96F83D1000F0030001F00301884243
:1046C00001D001F0ABFC86F83F40B6F848002886E0
:1046D00001B22C46594501DDA4F830B0FDF738FC95
:1046E000A06840F48060A06096F83810052993D146
:1046F00040F01000A06002208CE788F8004012E62D
:10470000706CB0F5437F02DA087806289BD1B9F8BF
:10471000061021F02001A9F80610FDF72FFE042055
:1047200078E70878062802D088F80070FBE50C4985
:104730000920087005206DE70348847003480C7059
:1047400080F856406DE600003C0400206000002028
:104750008C080020FE060020240A002064080020A7
:104760005402002030B585B001210420FFF7DEFBA4
:104770004FF40040ADF8100048208DF8130004A954
:104780001848FDF743FD01210846FFF7B7FB40F647
:104790008C20ADF8040003240020ADF80040ADF8F3
:1047A0000200ADF806004FF080456946284600F04B
:1047B000C5FF1C208DF80C008DF80D408DF80E40C3
:1047C00001208DF80F0003A8FFF778F801221146A9
:1047D000284600F08DFE0121284600F0BBFD05B003
:1047E00030BD000000080140704700002DE9F04195
:1047F000304CE07800285AD12078002857D0401E4D
:1048000010F0FF00207052D14FF49670208272B6E3
:10481000294F45F2AA50A7F872000020FDF776FB59
:10482000264D13202860FDF783FBA8BB3420E860E9
:1048300002202861224E6E61286940F04000286104
:10484000FDF776FB40BB00211E4A08465FEA255370
:1048500012F800C0BCF1FF0F00D00121401C80B253
:104860009842F5D3C1B9C4E9067639260127A06973
:1048700010F8011B10F8012BA061E06901EB022187
:1048800002886A612F6120F8021BE061FDF750FB8E
:1048900010B9761EB6B2EAD20120FDF737FB62B638
:1048A00001F010FC0848816821F480418160BDE876
:1048B000F0810000EC060020680C0020002002407F
:1048C00000FC000800FC000898020020194801685C
:1048D00041F010010160016821F0030101600168ED
:1048E00041F0020101601448416841604168416043
:1048F000416841F480614160416821F47C1141606C
:1049000041680E4A11434160016841F080710160C5
:1049100001688901FCD5416821F0030141604168CB
:1049200041F0020141604168C1F381010229FAD1DD
:1049300070470000002002400010024000002808DC
:1049400030B5044C039D6080A180E28023816581A5
:1049500030BD0000040A00200A44824201DA10B28D
:104960007047C91A8142FBDD08B270472DE9F04358
:104970004348DFF81081DFF81091C17F457A046861
:1049800001260023414A424880292BD301F01F0110
:1049900058F821100C420146096802D041F48051B8
:1049A00001E021F480510160CF0417D48F0415D5A4
:1049B000977AFF0707D0538199F800C02CF0020CBA
:1049C00089F800C00AE090F84670BFB14FF0020CC1
:1049D000012F18D080F8463080F81AC10F0B67F30A
:1049E0004D310160802D2AD305F01F0158F82110A8
:1049F0000C4201680CD041F004010BE080F84660E5
:104A000080F81A31EAE780F846C080F81A61E5E7D5
:104A100021F0040101604C070DD44C050BD5947AAC
:104A2000E40708D0538199F8005025F0020589F871
:104A30000050C0F898308C0864F38A210160917AA4
:104A4000C90717D1134991F86410012912D11249ED
:104A5000496C32290CDC0178490709D5018909051F
:104A600006D4D0F8981047F23054A14204D95681A8
:104A7000C0F89830BDE8F083491CC0F89810F9E7F9
:104A8000CC0500202C910008C6050020100A00204B
:104A900098020020680C00203C01002010B5FCF7B3
:104AA00067F90F48018821F0020101800C49183193
:104AB00009880C4A928E1144094A343211800849FF
:104AC0000C390A8842F001020A80011D0A884FF65B
:104AD000ED531A400A80018841F01201018010BD97
:104AE0000C0400403C04002006480188491C89B29F
:104AF0000180B1F57A7F04D34188491C41800021AF
:104B000001807047100700200F4810B5016841F080
:104B10000101016041680D4A1140416001680C4A81
:104B200011400160016821F480210160416821F495
:104B3000FE0141604FF41F018160FFF7C7FE054988
:104B40004FF00060086010BD001002400000FFF848
:104B5000FFFFF6FE08ED00E02DE9F0412F4D28881B
:104B60004FF00004000629D5FCF782FA2C4A2D48A4
:104B700007231778C8262C49012F22D02B4FB7F8CE
:104B800006C0BCF1000F3ED0B0F80CC04CF0080CD1
:104B9000A0F80CC0B0F806C02CF4006CA0F806C059
:104BA000886820F004008860FC801370CE870020A5
:104BB0004FF49661401C80B28842FBD32C80BDE844
:104BC000F0811B4F97F800C0BCF1010F0FD0BCF172
:104BD000020F11D0B0F806C04CF4006CA0F806C06B
:104BE000886840F00400886005203870DDE7B0F880
:104BF0000CC04CF0080C03E0B0F80CC04CF0100CEA
:104C0000A0F80CC0F0E70B4F3C70C78847F4006772
:104C1000C780886840F004008860C6E7102C014017
:104C2000EF060020100A0020980200202009002032
:104C3000F00600200D070020704700002DE9F0432A
:104C40004FF08040018A21F001010182AC480078D8
:104C500000287CD1AB4FF87B002878D1AA48406C63
:104C6000322874DCA9488068DFF8A4924104A94D79
:104C7000B9F804004FF0000403D4401CA9F8040064
:104C800028E1002874D02978012611B1012912D019
:104C900017E14946B0F5BE7FFAD92E70CC718C7100
:104CA000EC702C72287A0A18401CC0B21472287258
:104CB0000F28F7D305E1B9F802204946824201D90D
:104CC000EE7100E0EC7192488A7908300F2A15D213
:104CD000CB79082B0BD2C3F10708EB7912F800C08F
:104CE00003FA08F363441354CA79521CCA71CA798F
:104CF000082A03D18A79521C8A71CC7199F806105E
:104D0000C8460F2973D10D21FCF71CF9A881010AAF
:104D10006970C0B2A87088F8064098F816208A42D8
:104D200065D198F81510814261D198F80BC07A4985
:104D3000032302227948BCF1000F10D0BCF1010F0F
:104D400002D0BCF1020F14D080F86A2000E0CBE062
:104D500091F800C02CF00C0C0CF1080C0FE080F85E
:104D60006A6091F800C02CF00C0C0CF1040C06E009
:104D7000A9E080F86A3091F800C04CF00C0C81F882
:104D800000C098F80C10B6EB111F04D180F86E40EB
:104D900087F846400EE0B2EB111F04D180F86E6038
:104DA00087F8466006E0B3EB111F03D180F86E2050
:104DB00087F846200B0717D001F00F01012901D019
:104DC000022915D080F86C602C7198F80D102A79A2
:104DD00006FA02F30B406B71082A44D2DFE802F0B6
:104DE0000B124319242F363D80F86C40ECE768E045
:104DF00080F86C20E8E713B180F8704033E080F869
:104E0000706030E013B180F850602CE080F85040C2
:104E100029E023B180F8656087F8036123E080F81A
:104E2000654087F803411EE023B187F8F54080F81C
:104E30004D4018E087F8F56080F84D6013E013B13D
:104E400080F868600FE080F868400CE013B180F8EB
:104E5000666008E080F8664005E013B180F867609E
:104E600001E080F86740521CD2B22A71082AAED302
:104E700098F80E102A4A8B0705D587F8F16080F85C
:104E80006460568104E087F8F14080F86440548102
:104E9000C90702D080F8294001E080F8296098F81D
:104EA000111000F86D1FC2781E48012A1ED001B3F0
:104EB000012921D04FF48051A0F876101A493C20E6
:104EC0000870A9F80240A9F80440B9F80210491C7A
:104ED000A9F80210B9F80210B1F5FA7F04D940F22E
:104EE000F511A9F802102C70BDE8F08344F21C7192
:104EF000E2E74FF40051DFE741F25551DCE70000F3
:104F0000EF060020980200203C0100200010014024
:104F1000500C002088060020B4040020680C0020FB
:104F2000100A00201C050020EC0600202DE9F05F8F
:104F3000FDF724FA8E4D2888A5F10406C0070AD093
:104F4000308820F008003080288820F00900288070
:104F500001F0A0FDD9E02888DFF81892DFF8188268
:104F6000864C80071AD5B9F8001041F00101A9F864
:104F70000010B8F8000080491431503008802888AB
:104F80004FF6F95108402880308840F00400308006
:104F9000FFF738F884F83C00BDE8F09F2888784F88
:104FA0004007288871D520F004002880FFF72AF8F0
:104FB00094F83C108142EFD1308820F0040030801A
:104FC000FDF7B4FB2078410605D594F84C1094F811
:104FD0003B209142E0D03978400621F0020139703F
:104FE00004D5FEF7CFFA97F82F7004E094F83C0050
:104FF000FDF716FA0746DFF880B140F68C2A0BF170
:10500000180B062F47D294F83800B8423ED03846E5
:10501000FDF78AF92078C00716D094F83A0094F882
:10502000391000F00302914206D0A17A00F001008D
:1050300001F00101884215D1FDF7E0FAFBF7E4FE2B
:10504000FDF708FC384689E0FDF7D8FAFBF7DCFEEF
:10505000FDF700FC3846FDF7F1FA207840F001003A
:10506000207099E7288820F008002880206B8108AC
:1050700001EBD000504515D2B8F800100844ABF849
:105080000000308840F0080003E00DE0308820F098
:105090000800308080E7B9F8001041F00101A9F85C
:1050A0000010DFE75046E7E70007288831D520F0F9
:1050B00008002880308820F008003080FEF7A2FF2A
:1050C00084F83C00FDF732FB387820F0020038709D
:1050D0002078400604D5FEF755FA97F82F5004E0E3
:1050E00094F83C00FDF79CF90546062D08D294F88B
:1050F0003800A842B5D0FDF781FAFBF785FE2AE01B
:105100002048C18841F04001C180BDE8F05FFDF753
:1051100081BBC006288825D520F010002880308863
:1051200020F01000308097F838000C2802D2401C84
:1051300087F83800387840F002003870FEF722FA1D
:1051400097F82F50787884F8390094F83800A842FE
:1051500087D0FDF753FAFDF77DFB2846BDE8F05FE9
:10516000FDF76CBA4EF2BE110840288014E700002B
:105170001004004000040040240400403C010020D2
:105180003C040020100A00202DE9F04F514F85B05B
:10519000388820F0010038804E4800261030068004
:1051A0004D4CDFF838A14FF0010894F85C0042F64E
:1051B0003029C10774D072B64948816941F4007141
:1051C0008161816941F4806181614FF40040FEF7A3
:1051D0007FFE444D00212846FBF774FB0021284642
:1051E000FBF766FBDFF800B100215846FBF760FBD8
:1051F00000213E48FCF70AFA2846FBF77FFC584698
:10520000FBF77CFC4FF46020CDE902068DF80560C9
:1052100000968DF810808DF8048069462846FBF7CB
:10522000FFFC01231A460F212846FBF74AFD012106
:105230002846FBF73DFB00204946401C80B28842CF
:10524000FBD328462E600121FBF77AFD28688007F2
:10525000FCD524484C30006894F85C1021F0010122
:105260002144A1F85000FBF737FB62B6FEF796F831
:1052700047F69061AAF8001094F85C00401CC0B298
:1052800084F85C000C2822D212491431A1F8008065
:10529000388840F00100388005B0BDE8F08FFFE7A6
:1052A000134920F00100085A12490880114945F6B7
:1052B0005800083908800F4847F25801001F018044
:1052C0000C4920200C390880AAF80090D4E703206C
:1052D000A070E1E7000800403C0400202C080040DA
:1052E0000010024000240140002801400800024054
:1052F000E88C0008202C01400029018802D041F0F0
:10530000800101E021F080010180704710B50A881A
:105310004B88CC881A438B8823431A430B891A4342
:105320004B8989891A430A43A0F8442010BD002103
:10533000018041808180C1800181418181817047EC
:105340000029818802D041F0010101E021F0010132
:10535000818070470029018802D041F0010101E0FD
:1053600021F0010101807047002930F8441F02D06C
:1053700041F4004101E0C1F30E01018070470000DB
:105380004B4910B5884202D10121C41486E0B0F126
:10539000804F09D0474988420DD101210220FEF7F4
:1053A000B9FD0021022064E001210846FEF7B2FDAC
:1053B000002101205DE04049884206D101210420FE
:1053C000FEF7A8FD0021042053E03C49884206D1A5
:1053D00001210820FEF79EFD0021082049E0384900
:1053E000884206D101211020FEF794FD00211020F3
:1053F0003FE03449884206D101212020FEF78AFD92
:105400000021202035E03049884202D10121441496
:1054100044E02E49884202D10121CC043EE02C49CF
:10542000884202D101210C0538E02A49884202D184
:1054300001214C0532E02849884206D10121402053
:10544000FEF768FD0021402013E02449884206D180
:1054500001218020FEF75EFD0021802009E0204927
:1054600088420AD1841501212046FEF753FD002110
:105470002046BDE81040FEF74DBD1A49884202D1D2
:1054800001210C040AE01849884202D101214C0490
:1054900004E0164988420AD101218C042046FEF717
:1054A00051FD2046BDE810400021FEF74BBD10BD68
:1054B000002C01400004004000080040000C0040A7
:1054C000001000400014004000340140004C014036
:1054D000005001400054014000180040001C0040F2
:1054E00000200040004001400044014000480140CD
:1054F000002A828901D00A4300E08A4382817047F2
:1055000030B5028C22F001020284028C8388048B65
:1055100022F0020224F073050C882C430D891543F8
:105520004A882A43114DA8420BD0114DA84208D0F9
:10553000104DA84205D0104DA84202D00F4DA842F0
:105540000DD122F008054A8923F440732A4322F042
:1055500004058A882A438D891D43CB892B43838088
:105560000483C9888186028430BD0000002C01407C
:105570000034014000400140004401400048014027
:10558000028B22F008020A430283704770B5028C36
:1055900022F010020284028C8488038B0D8823F48D
:1055A000E6464FF6FF7303EA052535430E8922F0E0
:1055B000200203EA061616434A8803EA021232431F
:1055C000104EB04202D0104EB04215D122F08006EB
:1055D0004A8924F4406403EA0212324322F040066E
:1055E0008A8803EA021232438E8903EA860626433A
:1055F000CC8903EA8404344384800583C988018705
:10560000028470BD002C014000340140028B4FF633
:10561000FF7322F4006203EA012111430183704702
:1056200070B5028C22F480720284028C8488838B91
:105630000D8823F073031D4322F400730E894FF687
:10564000FF7202EA06261E434B8802EA0323334315
:10565000104EB04202D0104EB04215D123F4006675
:105660004B8924F4405402EA0323334323F4806635
:105670008B8802EA032333438E8902EA0616264307
:10568000CC8902EA0414344384808583C9888187E5
:10569000038470BD002C014000340140828B22F055
:1056A00008020A438283704770B5028C22F480524C
:1056B0000284048C8288838B0D8823F4E6464FF69F
:1056C000FF7303EA0525354324F400560C8903EAE9
:1056D000043434434E8803EA06362643094CA0427C
:1056E00002D0094CA04205D122F480448A8903EA01
:1056F0008212224382808583C988A0F840100684E4
:1057000070BD0000002C014000340140828B4FF638
:10571000FF7322F4006203EA012111438183704781
:10572000018582827047828822F07002828082889E
:105730000A4382807047A0F84010704730B5028855
:105740001B4B1C4C98420DD0A0420BD0B0F1804FA7
:1057500008D0194DA84205D0184DA84202D0184DC6
:10576000A84203D122F070054A882A43154DA84269
:1057700006D0154DA84203D022F44075CA882A43AA
:1057800002808A8882850A88028598420AD0A042CF
:1057900008D00E4A904205D00D4A904202D00D4AE0
:1057A000904201D1097A01860121818230BD000039
:1057B000002C01400034014000040040000800407B
:1057C000000C004000100040001400400040014068
:1057D00000440140004801404FF6FF7181800021E4
:1057E0000180C1804180017270470029018802D088
:1057F00041F0020101E021F002010180704700291F
:10580000018802D041F0040101E021F0040101808F
:1058100070470000204810B590F82010026801F091
:105820001F001E4951F820001D490242086802D09D
:1058300040F4803001E020F48030086019484FF0D7
:10584000000280794106184824D4184903880C883E
:10585000E31A9CB201230F2C08D30C8804808468BF
:10586000042C03DD124C2478022C05D0427F012A3F
:1058700006D00988418010BD4377C2770A884280EC
:1058800042880988891A89B240F21A629142F2D399
:10589000C37710BD427710BDCC0500202C910008C5
:1058A00098020020100A0020300C0020F80600208A
:1058B000EF0600202DE9F04FDFF8B8B16A48DFF8B5
:1058C000AC91DFF8ACA190F80EC0BBF91A70BBF92F
:1058D0001C60BBF91850BBF96C10BCF1070F48D223
:1058E000DFE80CF08D041A30485E7600D9F800200D
:1058F0008284DAF80020C284828CC38CA7EB8202F7
:1059000012B2A6EB83034A431BB2594342F3CF22A0
:1059100041F3CF23D11870E0D9F800204284DAF89F
:105920000020C284428CA5EB820213B2C28C4B438E
:10593000A6EB820212B243F3CF24514341F3CF23AB
:10594000E11814E0D9F80020C284DAF8002042847B
:10595000C28C438CA6EB820212B2A5EB83031CB26D
:105960004A43614342F3CF2341F3CF2419194942FB
:105970000AB244E0D9F800208284DAF80020428498
:10598000828C438CA7EB820212B2A5EB83034A43BD
:105990001BB2594342F3CF2241F3CF24111914E033
:1059A000D9F800204284DAF800208284428C838C6B
:1059B000A5EB820212B2A7EB83034A431BB242F368
:1059C000CF24594341F3CF22A11849420BB216E02C
:1059D000D9F80020C284DAF800208284C28C838C3B
:1059E000A6EB820212B2A7EB83031CB24A4342F336
:1059F000CF23614341F3CF22991849420CB2BBF93E
:105A00001E50594605F21E56A64201DACE8306E024
:105A1000A5F21E55A54201DDCD8300E0CC83B1F98E
:105A2000204004F21E55954201DA0D8406E0A4F2EE
:105A30001E54944201DD0C8400E00A84B1F9222056
:105A400002F21E549C4202DAABF8224008E0A2F2B5
:105A50001E529A4202DDABF8222001E0ABF8223060
:105A6000417B8173BDE8F08F980200203C24014007
:105A70003C2801401C0500202DE9F04704465C4805
:105A80005D4D002602785B48022AB0F9301004D040
:105A9000082A70D0092A6FD0A5E0C27B022A02D161
:105AA000B0F840204AB1E18769810423B5F90810B4
:105AB0001A460020FEF750FF8CE05049DFF8408185
:105AC000496A0F14E7808068410210D5B4F90200DA
:105AD00040F2DA21884269DD40F26A4188423FDCC7
:105AE000A0F2DA20FAF79BFC0022464B4DE0C0F30F
:105AF000C001C0F30020DFF8109181420CD1D8F82A
:105B0000440040F2BA41884250DD40F66A118842B2
:105B100026DCA0F2BA4034E03C480078C0060CD540
:105B2000D8F8440041F2243188423FDD41F2D4717B
:105B3000884215DC00F6DC4021E0354890F8701012
:105B4000012903D090F86F0001282FD1B4F9020089
:105B500041F6C811884229DD41F6786188420CDDA2
:105B60000823B4F93E101A460020FEF7F5FEE08740
:105B7000002819DB1BE02FE033E000F5C760A0F53B
:105B80000050FAF74CFC00224B46FAF7B4FB0E2209
:105B9000FAF720FCFAF77AFC00B2C0F580407843AF
:105BA0008013E087002F02DCE68700E0E787E08FC4
:105BB000184FE880D8F844107964A7F84C0000F03A
:105BC0007DFBB7F84E00688198F80A000028388FEE
:105BD00000D14042288106E00F48B0F87400688187
:105BE00000E069812E8184F83C60BDE8F087000008
:105BF000EF06002098020020600000201C05002015
:105C00003C0100200000794000C09240D0060020F6
:105C1000680C0020B4080020240A00202DE9F0417F
:105C2000B1F9025000232B241522854203DAB1F981
:105C30000000BDE8F081B1F9AE50854202DDB1F956
:105C4000AC00F6E701EB8205B5F90250854201DDB3
:105C5000134600E01446E21852085D1CAA42F1D136
:105C600001EB8206B6F90230834206DA36F9025CAD
:105C700036F9044C31F9221006E01D4631F9224074
:105C8000B6F90630B6F90410401B091BC617891176
:105C9000B60346EA90468703A1FB070CCA1702FB2E
:105CA00007C201FB06215A1BD317FAF73DFA000A77
:105CB00040EA0160001900B2B0F5804FB9DB43F64D
:105CC000FF70B6E770B5134C40F2244529462046D4
:105CD00000F03EF800281BD0204600F0C7F8294607
:105CE000204600F01DF80C4C00212046FBF78EFCEE
:105CF0002046FBF709FDC0F164000849C0B2042842
:105D0000087201D900F046F9BDE87040FBF742BDCA
:105D100070BD0000003801405800024058060020C5
:105D20000A0A01219140C9430180704700298189F5
:105D300002D041F4005101E021F40051818170470B
:105D4000002A828A01D00A4300E08A438282704797
:105D500030B501F01F0201240025C1F3421304FAFB
:105D600002F2012B0FD0022B0FD0838A4FEA1121B0
:105D70000088134204FA01F400EA040001D000B1E3
:105D80000125284630BD8389F0E7038AEEE710B588
:105D9000C1F3421301F01F040121A140012B07D0E0
:105DA000022B07D01430002A026805D00A4304E011
:105DB0000C30F8E71030F6E78A43026010BD0000AF
:105DC00030B50446008A85B00D464CF6FF71084098
:105DD000E98801432182A1894EF6F3100140A88889
:105DE0002A8910436A890A431043A081A08A4FF68A
:105DF000FF410840A9890143A1826846FEF7AEF839
:105E00001948844201D1039800E00298A18909044D
:105E100000EBC00101EB0010296801D5490000E04A
:105E20008900B0FBF1F06422B0FBF2F109010B092B
:105E30006FF018056B4300EB8300A3891D044FF03E
:105E4000320306D503EBC000B0FBF2F000F0070010
:105E500005E003EB0010B0FBF2F000F00F00084388
:105E6000208105B030BD0000003801408088C0F3BB
:105E700008007047F8B501210920FEF757F8012105
:105E80008803FEF753F810258DF803502020ADF855
:105E900000001A4E03248DF8024069463046FCF794
:105EA000B5F916490C31086820F020000860182068
:105EB0008DF803004020ADF800008DF802406946DF
:105EC0003046FCF7A3F948208DF803008020ADF898
:105ED000000069463046FCF799F98DF80350280117
:105EE000ADF800008DF8024069463046FCF78EF9A7
:105EF00001210420FCF7DCF9F8BD0000000C014092
:105F000030B585B0FFF7B6FF00244FF4E1300090C4
:105F1000ADF808400C201D4DADF80440ADF80A0066
:105F2000ADF80640ADF80C4069462846FFF748FF3B
:105F300025208DF8100004208DF811008DF81240F6
:105F400001208DF8130004A8FDF7B8FC012240F2EF
:105F500024412846FFF71BFF01212846FFF7E6FEF4
:105F6000FBF742FC012280212846FFF7E9FE0122CF
:105F700040212846FFF7E4FE012202210448FBF7F6
:105F8000D7FBFBF731FC05B030BD00000038014005
:105F90004400024070B51D4D00242878432834D1B8
:105FA0006878462831D1A878502807D0512805D0E4
:105FB000812803D0892801D0212826D1144E707160
:105FC000E9787172A81C891CFAF7F4FFB072717A33
:105FD000294409793182884217D106F10E000178EF
:105FE00041F0020101700B48016841F0200101609D
:105FF000317A0948002204E02B5D03552A55641CC0
:10600000E4B28C42F8D38078707170BD84070020B0
:10601000580600200C0C01409A0B002070B51D2082
:10602000FDF72BFCFDF7AEFA1D20FDF73CFC1548F3
:1060300090F82F10144D0623144C85F8381090F862
:106040003B1095F83B201143012A04D0022A07D0C7
:10605000042A0AD010E0827A8A420DD0007B09E03F
:10606000027D8A4208D0807D04E0827F8A4203D08C
:1060700090F82000884200D12370002085F840006D
:1060800070BD00003C0400203C010020EF06002011
:106090000B4800214180A0F1B0018A898280CB8920
:1060A0001A44C2800B8A1A4402814B8A1A444281E4
:1060B000898A1144818143F6FF71C18170470000D4
:1060C000EC010020084940F61C72B1F90C00904226
:1060D00002DA00F59F7005E041F2E302904201DD33
:1060E000A0F59F70C88170476000002038B5134844
:1060F000C16941F00401C1611E208DF80000022039
:106100008DF801008DF8020001248DF803406846E7
:10611000FDF7D4FB0A4984200880094947F69060BE
:106120002C3108800020091F0880054914310C809B
:10613000091F0880081F048038BD000000100240BD
:106140000008004030B420491E4A45788B7A114639
:1061500092F83B4091F83910AC4218D14BB1037919
:10616000994202D04379994201D140791AE080796D
:1061700009E08379994202D0C479A14202D182F820
:106180002F3011E0407982F82F0030BC7047C5787D
:10619000AC42FAD16BB1C379994202D0037A9942E9
:1061A00005D1007A82F82F0030BCFEF777BC407A28
:1061B000E9E7437A9942E2D00479A142DFD0007A3C
:1061C000E1E700003C0400203C010020FEE7000065
:1061D0002DE9F0470446007F012868D13548E18861
:1061E0000288511A89B2072916D30088E080B4F9D1
:1061F000000044F2DD414843401346F6D96148436C
:106200008013A060401000B2A0814FF08051B1FB1C
:10621000F0F0FAF7FFF82061B4F90C6096B1B4F928
:1062200002104DF6B05048430014A082B4F9047037
:106230004DF6B05207FB02F24FEA2245E58204D444
:10624000024603E00020E08330E0424212B22283A3
:10625000002D01DB2B4600E06B421BB2DFF85890AB
:10626000638398464FF4804AB24208DAFAF7C9F8D5
:106270002169F9F79CFFFAF7F0F8801304E0002990
:1062800001DA484600E05046E083B04509DA284686
:10629000FAF7B7F82169F9F78AFFFAF7DEF8801301
:1062A00004E0002F01DA484600E050462084BDE8B3
:1062B000F0870000F806002000C0FFFF10B5284856
:1062C000294C01782748022905D1C17B022902D136
:1062D000B0F8401029B1008EA4F84E0000202087AD
:1062E00010BD90F8462020482049022AB0F844000A
:1062F000097800B2C1F3810103D0012A0CD01C49F6
:1063000013E0012904D0022904D019496C390CE0AA
:1063100018490AE0184908E0012904D002291CD0D4
:1063200015496C3101E013496C31FBF7BFFD0E4993
:10633000A4F8400080B2483101F060FAB4F94C0092
:10634000B4F94A2041425143891324F8381FB4F963
:10635000101048438013E08210BD07496C39E4E710
:10636000EF06002098020020B4080020B4040020AA
:10637000CC8A000844880008888900080348002166
:1063800080F82A10C183018770470000B4080020FC
:1063900010B504000B462D4AC3F1000028D5644215
:1063A000002B12DAA04207DA214600F027FA32F871
:1063B0001000C0F5404041E00146204600F01EFAC2
:1063C00032F8100000F5004038E0A34208DA214618
:1063D000184600F013FA32F8100000F540402DE0A6
:1063E000204600F00BFA32F81000C0F5803025E0AE
:1063F000002B12DAA04207DA214600F0FFF932F84A
:10640000100000F5804019E00146204600F0F6F942
:1064100032F81000C0F5004010E0A34208DA21462F
:10642000184600F0EBF932F81000C0F5804005E0A6
:1064300053B1204600F0E2F932F81000B0F5004FF9
:1064400001DDA0F5803010BD002010BDF48C0008E7
:1064500040438013494300EBA13000220302002B8C
:1064600014DDB3F5001F01DC802001E04FF4005083
:1064700093FBF0F1014401EBD1714910814206D048
:10648000521CD2B20846062AF2D300E00021C8000E
:1064900000B2704702E008C8121F08C1002AFAD1F2
:1064A00070477047002001E001C1121F002AFBD194
:1064B000704700002DE9F047A44CA54821880288C8
:1064C000511A89B20F297DD30088A4F13C052080A0
:1064D000288F08B1401E28872B789E4AC3F381007D
:1064E00001281DD0022820D0D18B98489A4FDFF880
:1064F0006C92407E0026B1F5926F1DD8142819D3F6
:1065000078206076F88840F01000F88040F26660ED
:10651000A88123F001002870D67389F8006015E087
:10652000D08B00EB4000C00302E0D08B8C49484385
:10653000010CDAE7401C04E0B1F5DB6F06D310B1C3
:10654000401E607602E043F001002870B5F90200B9
:10655000B5F914304143C3EBC303C1F38F31C3F327
:10656000D10303EB510109B2A9829046D28B4FF0BF
:1065700080535043B5F91620C0F38F30C2EBC202EE
:10658000C2F3D10202EB500000B2E882AA6A424391
:106590001213EA6293FBF2F22A63724A1080A26835
:1065A0000A44A260E1680144E160207C401CC0B262
:1065B0002074072806D942F3CF002883C9106983C5
:1065C000E66000E0BFE0A66041F6C801267488429C
:1065D00004DD298B644AB2FBF1F1E981C11789031B
:1065E00041EA9041800342F69B420023F9F79CFD6B
:1065F000A88456482A78A0F13C005C49B0F906000E
:10660000930700FB01F14FEA2141C2F3810215D546
:10661000012A07D0022A0BD04FF2685141430914D6
:10662000A18011E049F68C4250430014A0801FE085
:106630004CF6183141430914A18025E0012A0DD000
:10664000022A17D0A0806984494948430014E08396
:10665000FBF74CFA47480088C0B143E04AF65C3289
:1066600042431214A2804BF62C225043001468843B
:10667000E183EDE74DF2AC5141430914A1804EF2A4
:106680007C414143091469843B49DEE795F82000C9
:1066900000BB88F80F6089F80060B5F91A00A0F512
:1066A0000C519F39B1F56E7F18D8617FF42912D94A
:1066B0003249E8802E4AA1F8460050430014A880D1
:1066C000A1F84400FF2085F8200081F828002C491B
:1066D0003C20087006E0491C617703E0607F08B148
:1066E000401E6077B5F91A10B4F91E0081420EDD24
:1066F000A07E7D2809D9F88840F00800F88021485C
:10670000017821F0020101700EE0401C06E0A0F2C9
:106710003D10814208DAA07E10B1401EA07603E051
:10672000F88820F00800F880B5F91810606908446E
:106730006061217E491CC9B221761F2903D940110D
:10674000A88366612676BDE8F0870000F00400208B
:10675000F806002098020020100A0020EF06002012
:1067600030330100C409002074E8260BCC0E010070
:1067700048850100FA060020D0450100680C002081
:10678000EC060020C6050020024941F68B308862E5
:1067900070470000B404002070B5164C0625207820
:1067A000062825D2DFE800F003080E141A2112484B
:1067B000FAF73EFC012016E00F48801DFAF738FC7E
:1067C000022010E00C480C30FAF732FC03200AE0FB
:1067D00009481230FAF72CFC042004E0064818306F
:1067E000FAF726FC0520207070BDFAF741FC2570F1
:1067F000257070BDF0060020388B0008090A05D00E
:10680000B0FBF1F0FF2800D9FF207047002070474F
:10681000D0E90021C368521A5A4301EBA2318160CA
:1068200041607047B0F90020B0F90210B0F90630AD
:10683000521A5A4301EBA231818041807047000017
:1068400030B5444B188844498A89801A85B2434838
:10685000434A0F2D047801F14C001DD31D888D8112
:10686000117A090713D5022C01D03E4912E03E4DA2
:10687000B0F90210B5F90050A94205DC02DA01F1C5
:10688000020108E0458007E0A1F1020103E0022CCB
:1068900002D1364909884180018F1D88691A89B261
:1068A0009C2942D319880187916A0023B1F5804F52
:1068B0002DDB2F49896CB1F5405F28DD2D4940F271
:1068C0006665B1F91010A94211DD43F69915A94288
:1068D00002DB40F2333108E040F23335A1F2666169
:1068E000694343F2333591FBF5F1818700E08387FB
:1068F0002149B2F806510978C1F381011DB1818F98
:1069000001F21E5119E092F84620022A0ED0838728
:10691000022C00D08387B0F95410B0F93C3001F15B
:1069200014029A420BDAA0F8542030BD012901D09C
:106930000229E4D1818F01F233318187E8E703F145
:106940001402914203DD1439A0F8541030BDA0F8B0
:10695000543030BDF806002014000020EF0600205F
:1069600098020020B2040020B0040020AC040020F3
:106970003C0100201C050020B40400202DE9FC414E
:1069800001210220FDF7BAFA01211920FDF7CEFA04
:1069900001213C48FBF78CFC4027ADF80070032434
:1069A0008DF802400420384D8DF8030069462846D2
:1069B000FBF72CFCE001ADF800008DF802401C2034
:1069C0008DF8030069462846FBF720FC4FF4E07180
:1069D0002846FBF7A2FCA815ADF800008DF8024090
:1069E00010208DF8030069462848FBF70FFC4FF490
:1069F000A060FCF795FF1D208DF8040001268DF89E
:106A0000056000258DF806508DF8076001A8FCF799
:106A100055FF1F498C2008801D494FF6FA702C3114
:106A200008806E20091F0880194814300680184815
:106A300008300780164920310D80154AD020121DDC
:106A40001080134A45F2F300183210800A1F45F2F5
:106A5000500010800E4A4FF6FF7038321080121D21
:106A60001080121D108041F21B10088000F012F8F7
:106A7000FBF7D0FE064810300580001F0480BDE8FB
:106A8000FC810000000C1A0000100140000C0140C5
:106A90000004004070B51D20FCF7E4FE2A4D4021A3
:106AA0002846FBF731FC840080212846FBF72CFCAC
:106AB00044EA4004A9152846FBF726FC0443E0B24B
:106AC000224C84F83C00FBF7ABFC0546052805D9B1
:106AD0001F48C18841F04001C18001E084F838506E
:106AE0001C48007A000703D594F838001A490D5C59
:106AF0004FF6FA702063E062A06260622062E0619B
:106B0000A0611648606300206064A06484F83F00C0
:106B100084F84000FBF732FCA07AFF2811D0022055
:106B200084F83D000E48008820662846FCF7D4F81B
:106B3000207820F001002070BDE870401D20FCF797
:106B4000A7BE0120ECE70000001001403C0100203E
:106B5000100A002098020020F8940008DCFF0500CD
:106B6000240400402DE9F0434E484F4902880B8829
:106B70009A1A92B20F2A69D3098801804B49098B6E
:106B8000027D00EB42029180017D491CC9B2017572
:106B900008295BD3002404752246017D00EB4103E4
:106BA000491CB3F90430C9B202EB630212B2017599
:106BB0000829F2D33E4904753E4B4A8044800E7842
:106BC0009D895FEAC67C40F638694FF0030714D010
:106BD000A2F22B5C42F6E858C44520D3A1F1020C86
:106BE00026F00204ACF8002047750C7040F22B54DC
:106BF000A24211DA45F004021EE046F001060E70D2
:106C00004A4507DD45F001029A8126F002020A702A
:106C1000477519E0447517E045F002020CE04A455B
:106C20000CDA8775427D12B1521E42750CE046F0B7
:106C300002020A7025F007029A8105E0B30703D526
:106C4000837D2BB15B1E837540888880BDE8F0830F
:106C500042F6AA239A4222DAB1F904302BB941F262
:106C6000CD05AA4201DA4480EEE7134C920302EB11
:106C7000843241F67244B2FBF4F214B240F233357E
:106C800002464480AC4200DA5580B2F90240E41A70
:106C900004F5A374B4F5237FD6D84380D4E74FF42A
:106CA0008043FAE79C0A0020F806002098020020A2
:106CB000C6050020100A0020C8F1FFFF2DE9F041B1
:106CC0006C4CDFF8B4E14FF0000594F82C10C807C5
:106CD00006D094F930104B42002956DD0E4655E09F
:106CE000664884F82F506587654A90F8380084F824
:106CF00038001586CEF80450CEF80850614E40F2A8
:106D00006663CEF80C50A4F8743036F810005E4E6E
:106D1000768830444FF6FF7606EA800024F8280B88
:106D20004FF080602060A320208460845810A084ED
:106D3000E38440F699102085580060854FF4805018
:106D4000A08541F23330E08541F26660208641F64D
:106D50009910608641F6CC40A0864FF40050E08642
:106D600042F23330208742F26660608742F6991023
:106D7000A08742F6CC40E08782F89D5041F00100A8
:106D8000207184F84450BDE8F0811E4694F92F002C
:106D90004242002801DD074600E01746F61B012E9F
:106DA0000BD0002800DB02465FFA82F684F8300040
:106DB00094F84700012805D041E0002900DA19467F
:106DC000CEB2F3E794F931305942002B01DB18467B
:106DD00000E0084694F93220C7B25042002A01DB95
:106DE000944600E08446BC4508DD002A00DA0246ED
:106DF000D7B2002B00DA0B46D8B207E0002B00DA3E
:106E00000B46DFB2002A00DB1046C0B204EB4000A4
:106E1000B0F9481004EB470030F9482F11444910ED
:106E2000018084F8475084F8365084F8355084F84F
:106E3000345084F8335084F8325084F8315004EBE5
:106E400046007546B0F948006087BEF80410C823B4
:106E500009B26422FDF780FD6860E968401AA968FC
:106E60000844A860B5F900104843C013E860A4F8CE
:106E7000740088E7240A0020B40500203C010020AB
:106E8000980200200A95000860000020F0B45448E1
:106E900090F82C10C90776D0524990F8383000226B
:106EA00091F838108B426FD04F4CA0F86A204F4DAC
:106EB000E65C04468E4294F92F4002D0EE5C8E428E
:106EC0000FD1641C64B280F82F40EB5C8B4202D17E
:106ED000641C80F82F4090F92F300F2B1BDD0F23FF
:106EE00017E0434DEE5C434D8E4202D0EE5C8E4285
:106EF00011D1641E64B280F82F40EB5C8B4202D14A
:106F0000641E80F82F4090F92F406FF00E039C42D2
:106F100001DA80F82F30324B90F83750313390F847
:106F20002F40EC5490F837305B1CDBB280F83730E0
:106F3000062B01D380F8372090F9314090F9333097
:106F40009C420ED190F93540A3420AD190F93240CB
:106F500090F934309C4204D190F93640A34200D1DC
:106F6000012280F847201F4A80F8381090F92F50EE
:106F70001378214A012D0DDD14465E07A46804D55F
:106F800044F0080403E028E015E024F008049460CD
:106F900080F82D10B5F1FF3F0ADA5B07936802D540
:106FA00023F0080301E043F00803936080F82D10FC
:106FB000F0BCFBF7E3B990F8471001290DD1B0F808
:106FC0006A1043F60953491C89B2A0F86A10994225
:106FD00003D9A0F86A2080F84720F0BC7047000071
:106FE000240A00203C010020EC940008F2940008E0
:106FF000FE940008049500089802002030B520494E
:10700000204AB1F86A301088C01A80B20F2836D3EF
:107010001088A1F86A001C4D00204FF000432A5C44
:10702000940903D00124B4EB921F24D1D20622D0BC
:10703000164A52F820201268134C123434F81040CB
:10704000224201EB000494F9722008D00A2A04DBE2
:107050000A6823FA00F4224308E0521C09E012F106
:107060000A0F05DC0A6823FA00F4A2430A6002E072
:10707000521E84F87220401CC0B21128CFD330BDFC
:10708000CC050020F8060020F8900008F8910008D0
:107090002DE9F00779497A480A8903889A1A92B249
:1070A000082A74D300880881A1F12C0042890AB112
:1070B000521E4281734A92F82820802A67D302F038
:1070C0003F020A70C2890AB1521EC281B1F906207C
:1070D000902A0CDB8A46FF2A09D08146C089002805
:1070E00055D1694800230078092805D005E0BDE89E
:1070F000F007624800F092B90823644A92F8EA5017
:107100000DB143F004036248817AC90701D043F00E
:107110000203D2F808C05FEA0C5101D543F0010325
:10712000176800215B4EFC0302D596F8654004B158
:107130008021C4885FEA446801D541F040015FEADC
:10714000845801D541F020015FEAC47801D041F0B4
:107150001001007A400701D541F008014E4800783F
:10716000C00701D041F00401A00601D541F00101A2
:107170000020012D00D1082096F8705085B992F8B2
:107180004620022A04D0012A05D03AB108E072E074
:1071900040F0030004E040F0020001E040F0010094
:1071A0007A0701D440F02000CCF3C0020025CCF3D4
:1071B000002C624502D13A0700D4042596F86F20CE
:1071C000012A01D145F00105344A0027BC46127856
:1071D0003E46C2F38102012A04D0022A04D0032AC7
:1071E00004D004E0022602E0042600E010262C4A27
:1071F00064060ED5214C1C342478240609D5147855
:10720000640606D4274A40F6CC44926D6243140CBF
:1072100005E0B2F8AE2040F699146243940B4FF0AB
:1072200008088AF80A804FF061088AF80B808AF80B
:107230000C308AF80D108AF80E008AF80F508AF880
:107240001070270A4B4083F06901414069408AF879
:10725000117079408AF81240614052468AF813C092
:1072600071408AF8146051754FF4C871A9F80E1076
:10727000FF20AAF80600BDE8F0077047B40600201A
:10728000F8060020CC050020EF0600209802002020
:10729000100A0020680C002008090020B404002017
:1072A0003C010020E80700204C48816941F0FC01C6
:1072B00081614FF4A060FCF733FBFBF739FBFCF76F
:1072C00093FCF9F773FCFCF789FAFDF74BFAFFF72B
:1072D00055FBFCF7C9F9FFF7DDFBFBF79BFA404DC7
:1072E0004FF40050A5F81601FEF70AFE00214FF4F6
:1072F000FA5340F2EE220020401C80B29842FBD3A9
:10730000491C89B29142F6D33648002680F8726053
:10731000F9F7E2FAF9F788FFFCF796FCF9F756FE61
:10732000FEF7E4FE102230493048F8F72EFF304CCB
:10733000314FE08820F04000E0802E48017821F0B5
:1073400020010170FA20F8814FF49670E887FFF76A
:107350001BFA2A492A48FCF7F4FB2A48FCF716FCDA
:107360002948416A88472948416B8847FFF706F852
:1073700027494220C8802749C8603E71E088E081E3
:107380002089208260896082FAF7B8FEFAF71AFE37
:10739000FFF790F8FFF7E6FB00F0F8F9FFF72EFE95
:1073A00000F0C4FFFEF736FAFAF770FCFBF7B2FC08
:1073B000FFF746FAFCF7A0FEFBF7D4F8FBF706F957
:1073C00000F07AF8FFF764FE1348FAF757FA00F076
:1073D0006FFAFDF70BFAFAF7BBFBCFE7001002409C
:1073E000980200201C050020680C00200C060020DC
:1073F000100A00203C010020EC0600208C08002030
:1074000064080020F803002034000020D000002091
:10741000140700202804002090090020F0B523491B
:107420000278B0F9064000231F4E31F81210FF2CED
:1074300018D0B0F904701E4DBC4231DA00EBE407FD
:1074400004F00704BF7AA7408478FFB23CB190F8FB
:1074500001C0ACF1010C64451FDA3C061DD455F89F
:1074600022200DE056F82220116012498A79521C20
:10747000D2B28A71022A02D38370C3808B71F0BDAD
:1074800011608178491CC9B2817042789142F6D36B
:107490008370C188491CC180F0BD56F82220EFE7F7
:1074A00055F822201160F4E7D89200080A910008EC
:1074B0008092000888060020F0B561486149B0F864
:1074C0006C200B889A1A92B29C2A7BD30988A0F868
:1074D0006C105D495D4F91F82A1001F0070297F892
:1074E0004610022A00D1491E594C80F83E104FF038
:1074F0000203E2884FF00001550401D5012236E075
:10750000A489E50601D5062231E0250701D5082228
:107510002DE0550603D44F4D2D78AD0601D504223C
:1075200025E0150501D5072221E0150601D50A221F
:107530001DE0950601D50C2219E0150701D50B2297
:1075400015E0550701D4D50501D510220FE0D50669
:1075500001D505220BE0650703D4A50701D4E40794
:1075600002D080F86E3007E0920403D5032280F841
:107570006E2001E080F86E10374A384C92F820E017
:10758000324A251FD2F808C02D4AB2F87060721C2A
:1075900092B2BEF1000F0DD02CF4000CC7F808C059
:1075A00090F86E70B7B11E2F1AD090F86F200AB302
:1075B00025E007E04CF40006BE60A0F870200A2A1F
:1075C00001D22360F0BD142A01D22B60F0BDA0F8D7
:1075D0007010F0BD2B60A0F8701080F86F10F0BD37
:1075E000642E04D2A0F87020322AEED3E9E7A0F886
:1075F0007010EAE77F1C80F86F70A0F8701090F8A8
:107600006F20012A10D0002AE9D0B0F87060761CF3
:10761000B6B2A0F870601E2ED7D323603C2EDED900
:10762000521E80F86F20D2E7B0F87020521C92B240
:10763000A0F870202360C82AD1D980F86F10C6E75F
:10764000CC050020F8060020680C002098020020DD
:10765000100A00203C010020B4040020141C01404A
:10766000F0B54248B0F84810491C89B2A0F848105B
:1076700002297AD33E490024A0F848400A783D4BBD
:10768000042A57D04FF48041082A0BD0A0F10C02F5
:10769000B2F900208A4200DA1146B3F980208A420A
:1076A00000DA1146344A92698A4200DA11B2418204
:1076B00082881D8AC2EB8502304D12B22D78C5F347
:1076C00081062A4D42F231667243B5F97650921224
:1076D0006A431213C26086681546C6EBC60642F3BB
:1076E000D102F60202EBA6328260C66C1644C66472
:1076F000B0F850707F1CBFB2A0F85070B7F5806F23
:1077000004D3B6120682A0F85040C464891A1C4EF5
:10771000C26A724340F255564E4302EB4602466A35
:1077200032444262B3F93030B2EB034F06DD1A0443
:10773000426206E01349B1F90410B3E7002A00DA07
:107740004462C162104990F83D2091F838108A4295
:107750000BD080F83D10B0F84210A0F84410B0F8FB
:107760004010A0F84210A0F84050F0BD1C050020C9
:10777000EF06002098020020000C0020B404002036
:10778000C3F5FFFF1C0C00203C01002017481849DE
:10779000B0F85A200B889A1A92B20F2A25D309887A
:1077A000A0F85A10134941F6515391F84D10CA07E9
:1077B00001464FF48042B1F9001059438913A0F8F3
:1077C0006C100D490B78A0F10C01022B06D1B1F918
:1077D0000030934202DA1B1D0B8000E00A8000217A
:1077E000A0F8601020F85C1F428070471C05002044
:1077F000F8060020680C0020EF0600204FF6FF720C
:1078000002EA800210F4404315480ED0B3F5804FD1
:1078100014D0B3F5004F4FEA122216D0C2F5807390
:1078200030F813305B424B8005E0120A30F812301A
:107830004B80C2F5807230F812000FE0120AC2F5D8
:10784000807330F813304B8005E030F81230C2F509
:1078500080725B424B8030F81200404208807047D3
:10786000F48E0008104A518A908AD28A1638463916
:10787000A2F1110200D54942002A00DA5242114415
:10788000002800DA40420844084943F6284300B281
:10789000B1F936205A43921340F2D733584302EBE2
:1078A000A030C88670470000980200201C05002008
:1078B000F0B5904990480A8903889A1A92B23E2AF4
:1078C0001ED30088088101F138004FF4FA63428A20
:1078D0009A4202D2521C428200E04382874A92F8C6
:1078E0002220802A0CD302F03F020A70B1F9062050
:1078F000402A06DBFF2A04D0C2883AB1521EC28059
:10790000F0BDBDE8F0407B48FFF788BD428A9A424F
:10791000F6D307784FF0010E3A074FF0FF055BD51D
:10792000847A40F2DC52630708D444F00403837283
:10793000C28081F80BE081F80AE04CE04378072B25
:1079400005D0032B03D0052B01D0062B07D16606EB
:1079500005D444F040038372C280052239E0654AB1
:107960005FEA437C02F138024FF42076127A0DD59B
:107970005FEAC26C0AD45FEA446C07D442F010029A
:1079800002723A0628D4C680192222E0DF0709D005
:10799000970707D4670605D442F002020272C68038
:1079A000042216E09F0709D5170707D4670605D4F8
:1079B00042F008020272C68003220AE01B070BD5C0
:1079C000530709D4630607D442F004020272C6804A
:1079D0000B22CA728A72CD80494AB2F92230B2F9BA
:1079E0001A7003F23D140022A74200DB0276414EDA
:1079F000444C06F13806A479B6895FEAC46C06F1F6
:107A000001064FF4C874B6B213D58681B6F57A7FF5
:107A100005D9017A21F0800101728281F0BD037ADB
:107A20001E06FBD4828143F080020272C4801120C2
:107A300035E09F4216DA037E052B13D28681B6F518
:107A4000487F04D98281027A22F040020272027ACF
:107A50005606E3D45B1C037642F040020272C480F7
:107A600002201CE0284B1C89C4F3C006C4F3002785
:107A700040F2EE24BE4216D11E78360713D4427E61
:107A8000012ACBD1428BB2F5167F02D2521C42831F
:107A9000F0BD827A42F002028272C4800F20C87266
:107AA0008872CD80F0BD93F80D714FF40046012F20
:107AB00018D1164F41F6583C7F6C674512DD83F8AC
:107AC0000CE1134B1E60C38AA34202D25B1CC3822B
:107AD000F0BD4FF4FA73C3801C23CB728B72CD8040
:107AE000C282F0BDC2820A4883F80C21001F0660E2
:107AF000F0BD000098060020F8060020CC0500200C
:107B0000B4040020100A0020980200203C0100204C
:107B1000140801402DE9F05FFC48FD49DFF8F4A3AB
:107B2000007E0A1D131D012850465AD030F85A4FC6
:107B30000C8041881180BAF85E001880FDF7BAFE0B
:107B4000F54DF64C49F2CD32B5F91E006083B5F91A
:107B5000201043F6CC4C00EB410151430914A183A2
:107B6000B4F92230B4F9206001FB03F200FB0622D5
:107B700042F38F326282B4F9167007FB0CF7BF1321
:107B800040F2333C714302FB0CF200FB131007EB95
:107B9000A232E28240F38F30A082B4F91810E04F95
:107BA000C1EBC10141F3D10101EBE000DD4E2083C7
:107BB000786C3060316930468847DB4930894880CD
:107BC0000846FDF759FFDFF8649301264FF0000BDC
:107BD00099F8000008280CD0618E218204284AD030
:107BE0001AE030F8604F0C8041881180BAF86400C8
:107BF000A3E7CF4890F92F10491C022939D890F8F3
:107C00006C1019B1B4F85200208205E0618E218217
:107C1000A4F8521080F86C60B4F91410B4F90A009A
:107C2000C44AF9F73BFCE062BAF91611884204DD58
:107C3000C048E162027B91404162B848DFF8F8E257
:107C40004C3847F2A30802784EF2461172B3012A6B
:107C500052D080F800B000BF99F8000004280DD081
:107C6000B44AB4F91210B4F90800283AF9F716FC2E
:107C700007E0608EC8E7686A0014E062B87A70B303
:107C8000AE48AF4DA0622860E06A68602846FCF705
:107C900099F8A84F287C3C3F01285ED0A06A386044
:107CA000A8480178C9075CD040695BE0B5F91E209F
:107CB00042448A4209D8B5F9202042448A4204D875
:107CC000B5F9222042448A42C6D9A0F802B0B7F8DA
:107CD000AE205946B2F5C87F02D8467007E039E0B9
:107CE000B2F5487F01D8022200E0032242708AF8F0
:107CF0000F1089F8001024E080F800B0B5F91EC01C
:107D00005A46C4448C4509D8B5F920C0C4448C45B2
:107D100004D8B5F9225045448D429DD9B7F8AE102C
:107D2000B1F5C87F01D8467006E0B1F5487F01D8AB
:107D3000022100E00321417042808AF80F2089F877
:107D40000020BEF8061041F40061AEF80610FAF704
:107D50002BF981E74FF4AF7093E768693860A86941
:107D600000E0E06A786073483C38FCF79FF96B4D9F
:107D70006A4935F8100F3C39FFF740FDDFF89C9158
:107D8000DFF8C481A9F14C09D9F81010C9F86C10BA
:107D9000B5F91010B868B5F9122000FB01F4FB68C2
:107DA000504303FB124444F38F3703FB010040F3BD
:107DB0008F34AF86EC86A8F802704546A8F80440D8
:107DC0004046FEF705FA287F09F11405012830D056
:107DD000604241104DF6B35047433A1469802A80FF
:107DE0008B18A9F80440A9F80630891AA9F80810D8
:107DF0008AF80CB0B9F90430D84654464946002BED
:107E000000DD2673B1F90600002802DD227B921CFA
:107E10002273B9F90820002A02DD217B091D217394
:107E2000217B072920D2DFE801F01F1B3419301D08
:107E30003200B8F920304DF6B352584240106880F5
:107E4000B8F91E10514309142980A9F804304318C9
:107E5000A9F80630401AA9F80800C9E7667303E0DC
:107E6000022100E003216173DFF8B090374E384FF4
:107E700099F800100129617B0DD0072945D2DFE870
:107E800001F0E7FEFDFCFBFAF9000421EBE7052118
:107E9000E9E70621E7E7072937D2DFE801F0D9044F
:107EA0001B627999AF0001461846FBF731FE286046
:107EB000B5F90200B5F9001043F2046201445143E0
:107EC000090C5043A4F85A10000CA4F85C00A4F864
:107ED0005E8027E1404201B2504200B2FBF718FE3B
:107EE0002860B5F9020043F204614143090CA4F88B
:107EF0005A10B5F90010084443F204614843000CDD
:107F0000A4F85C00A4F85E803AE1A1E090090020AA
:107F1000342C0140980200201C0500206000002045
:107F20003C01002028040020E8030020EF06002088
:107F3000240A00208C080020100A0020A2FEFFFF67
:107F4000E809002008090020C4090020002401409D
:107F5000002801403046F8F787FE01231A46072122
:107F60006BE019461046FBF7D3FD2860A4F85A8051
:107F7000B5F90200B5F9001043F20462014451431F
:107F8000090C5043A4F85C10000CA4F85E0026E134
:107F90005942404209B200B2FBF7BAFD2860A4F88A
:107FA0005A80B5F9020043F204614143090CA4F878
:107FB0005C10B5F90010084443F204614843000C1A
:107FC00039E13046F8F750FE01231A46052134E026
:107FD0001146FBF79DFD2860B5F9020043F20461EC
:107FE0004143090CA4F85A10A4F85C80B5F90010BC
:107FF000084443F204614843000C47E1504201B297
:10800000584200B2FBF784FD2860B5F90200B5F9CB
:10801000001043F2046201445143090CA4F85A10C1
:108020005043A4F85C80000CA4F85E005EE130468A
:10803000F8F71AFE01231A4606213846F8F714FE0F
:1080400001213046F8F786FD01213846F8F782FD18
:10805000B34EB9F808004D463080B9F80A00708078
:10806000B9F81000B0803046F9F754FCB4F85A0063
:10807000F18805E018E1ECE0BDE08EE05EE031E083
:108080000844A4F86000B4F85C0031890844A4F8FE
:108090006200B4F85E0071890844A4F86400317E7F
:1080A000A048012978D034F85A1F018061884180A6
:1080B000A18881809B49028808310A8042884A80D1
:1080C000808888809748896A0830884795F8360004
:1080D00000287DD0F8F7CCFF15F8360F401E287029
:1080E000BDE8F09F01461846FBF712FD2860B5F980
:1080F000020040F68151484380136880B5F90010B2
:1081000040F68152514389134218A2F681525242DD
:1081100052082980A4F85E201044A4F85C000844AA
:10812000A4F85A0000213046F8F714FD0021384623
:10813000F8F710FD01231A4606210BE7404201B271
:10814000504200B2FBF7E4FC2860B5F9020040F6AB
:108150008151484380136880B5F9001040F6815280
:10816000514389134218A2F6815252425208298083
:10817000A4F85E201044A4F85A000844A4F85C0057
:1081800000213046F8F7E6FC00213846F8F7E2FC1B
:1081900001231A460521DDE6B4E019461046FBF737
:1081A000B7FC2860B5F9020040F6815148438013BE
:1081B0006880B5F9001040F6815251438913421886
:1081C000A2F68152524229805208A4F85A2000E0B7
:1081D0009BE01044A4F85E000844A4F85C00002171
:1081E0003046F8F7B7FC00213846F8F7B3FC012316
:1081F0001A460721E5E65942404209B200B2FBF7B0
:1082000087FC2860B5F9020040F68151484380138D
:108210006880B5F9001040F6815251438913421825
:10822000A2F68152524252082980A4F85A201044E2
:10823000A4F85C000844A4F85E0000213046F8F77A
:1082400089FC00213846F8F785FC01231A460621EF
:10825000B7E61146FBF75CFC2860B5F9020040F672
:108260008151484380136880B5F9001040F681526F
:10827000514389134218A2F6815252425208298072
:10828000A4F85C201044A4F85A000844A4F85E0046
:1082900000213046F8F75EFC00213846F8F75AFC1A
:1082A00001231A460521C2E6504201B2584200B2EB
:1082B000FBF72EFC2860B5F9020040F681514843D7
:1082C00080136880B5F9001040F68152514389133C
:1082D0004218A2F68152524252082980A4F85C202A
:1082E0001044A4F85E000844A4F85A000021304667
:1082F000F8F730FC00213846F8F72CFC01231A4629
:10830000072194E634F8601FCFE607480088A0F5FF
:10831000D04168393FF4E4AEBDE8F05FF9F78ABDBB
:10832000900900202C000020182C01402DE9F0417C
:10833000904C9148B4F85A100288511A89B20F290A
:108340006FD30088A4F85A008C480088DFF8308288
:10835000C0074FF000054FF0010741D0874AD4E92C
:108360000C1024321388B1EB530F02D21288511A29
:1083700008444FF4F371884200D208468149B1FBAA
:10838000F0F0616CC1F35101084406466064F8F7EF
:1083900046F800227C4BF7F7AEFF4FF040427B4B94
:1083A000F7F7A9FF0E22F8F715F8F8F76FF8A4F819
:1083B000A40094F86500401CC0B284F86500082849
:1083C00034D36C4898F84620001F03789A4201D0B5
:1083D000027045806E4A13786E4A23B1458021E0D1
:1083E0006564A56458E0D8F89410A1F5FA618E424E
:1083F00011DD616D8B1C9E4205DDB0F902100A296A
:108400000DDA491C06E08E4205DAB0F902100029A7
:1084100008DD491E4180B0F902000A2802DB17700E
:1084200001E0A2E01570666584F865505A484FF483
:10843000A5420178C1F38101012949D002294AD01E
:1084400044F687712181A4F8A020B0F9243089B2C4
:108450004B439B13A4F89C30B0F90E0000237043EB
:10846000B0FBF1F0A16CC0F3D100C1EBC101C902B6
:1084700000EB9130A064F017810341EA9641B0030C
:10848000F7F752FEB4F8A210C1EBC101C902C0084F
:1084900000EB9130A4F8A200616CA06E0844A066C5
:1084A00094F86C20521CD2B284F86C20082A05D3B0
:1084B000C008A4F86E0084F86C50A566374A384EA0
:1084C000D388580633D498F80F00022806D02CE041
:1084D00043F20451B6E744F24621B3E7B06840F6F0
:1084E0009916B04221DD94F8380094F88660B042C5
:1084F0000CD084F8860094F83D0000F00106C0F32B
:108500004000864202D1A4F8825004E0B4F8820010
:10851000B0F5966F05D2B4F88200401CA4F8820032
:1085200005E043F08000D08001E0A4F882501148BB
:1085300094F83F20B0300C2A01D2C57400E0C77413
:10854000174B41F2482641F2504C93F83C400C4BFB
:108550000C2AB3F882300AD3B14208DB012C06D0D2
:10856000614502DD002B00D18774BDE8F081857480
:10857000FBE700003C010020F8060020000400405A
:10858000980200204564BD0100209C40133B33400D
:10859000E6030020E7030020B4040020100A0020B6
:1085A0001C0500202DE9F041384C394E394F207818
:1085B00041F23331C2074FF000050CD0A28962B3FB
:1085C00094F90700002800DA4042C0B2032829D2FB
:1085D00040F2AE702AE0A570E5732F4AE571A581DF
:1085E00092F83830237220F00800A18040F0020099
:1085F00020703D867560B560F560916C490005D0CE
:1086000041F68461A18140F010002070C0B240F0BA
:10861000010020706574BDE8F081658120F01000D4
:10862000207015E0042803D240F6510060810FE06D
:10863000052802D240F69910F8E740F6CC42062809
:1086400003D3072801D3082801D2628100E06181A9
:1086500097F89D0098B9B088102301B2B4F90A00C8
:108660003622FCF779F97060F168401AB168084465
:10867000B060B6F900104843C013F0603886388EF9
:1086800010B10120A070C6E7A570C4E71C0C002043
:1086900078060020980200203C0100202DE9F041DE
:1086A000554C2678F0077CD05448217A544D90F8E8
:1086B000380081427BD0534A2346DFF84CC1575CD7
:1086C00093F90E2093F90730874203D01CF801700C
:1086D000874213D146F002065B1C26705BB2E37141
:1086E0001CF80110814201D15B1CE37194F9071061
:1086F000062901DD0621E171521C1CE0434F17F8E9
:1087000001C0434F844503D017F801C0844513D1FD
:1087100026F002065B1E26705BB2E371795C814233
:1087200001D15B1EE37194F907306FF005018B42B4
:1087300000DAE171521EA273207294F907108A1CAC
:10874000042A02D941F68462A2812C4A01291278B6
:108750000ADD2B4B56079B6802D543F0080301E066
:1087600023F00803AB606070B1F1FF3F09DA5107F5
:10877000A96802D521F0080101E041F00801A960D3
:108780006070F9F7FBFDA078012810D121488068BE
:10879000A3280CDA94F90700022803DD0220E07117
:1087A00005E01EE06FF00101884200DAE171A08966
:1087B000002630B1401E0004000CA08101D1E671FA
:1087C000A673E87B04280CD0B5F930105123412260
:1087D0000020FCF7C1F82886002802D1E07B10B108
:1087E000A670BDE8F0810C4806700C480670207831
:1087F00020F001002070F4E71C0C00203C01002058
:1088000098020020EC940008F2940008FE940008FE
:10881000049500081C0500200C070020EF0600202E
:10882000743F713D9B3BED396238F436A1356534B8
:108830003F332A32273133304C2F722EA32DDF2CB9
:10884000242C722B000000361C070038AA0A003ABC
:10885000AA0A003CCC0C003ECC0C0040380E004272
:10886000380E0044380E0046380E0048380E004AD4
:10887000C711004CC711004EC7110050C71100525C
:10888000C7110054C7110056C7110058C711005A2C
:10889000C711005CC711005EC7110060C7110062FC
:1088A000C7110064C7110066C7110068C711006ACC
:1088B00000000036000000388E03003A8E03003CB2
:1088C000FA04003EFA0400401C0700421C07004462
:1088D0001C0700461C0700481C07004A8808004C7B
:1088E0008808004E88080050880800528808005404
:1088F00088080056880800588808005A8808005CD4
:108900008808005E880800608808006288080064A3
:1089100088080066880800688808006A0000003639
:10892000000000388E03003A8E03003CFA04003E3B
:10893000FA0400401C0700421C0700441C070046C4
:108940001C0700481C07004A8808004C8808004E95
:10895000880800508808005288080054880800568B
:10896000880800588808005A8808005C8808005E5B
:10897000880800608808006288080064880800662B
:10898000880800688808006A0000003A2202003C5B
:108990008E03003EB0050040D2070042AA0A004400
:1089A000CC0C0046EE0E00481111004A3313004C67
:1089B0009F14004E0B160050771700527717005483
:1089C00077170056771700587717005A7717005C0B
:1089D0007717005E771700607717006277170064DB
:1089E00077170066771700687717006A7717006CAB
:1089F0007717006E00000036000000388E03003A42
:108A00008E03003CFA04003EFA0400401C070042BA
:108A10001C0700441C0700461C0700481C07004AAE
:108A20008808004C8808004E8808005088080052CA
:108A30008808005488080056880800588808005A9A
:108A40008808005C8808005E88080060880800626A
:108A50008808006488080066880800688808006A3A
:108A60000000003A2202003C4404003E660600403A
:108A700088080042AA0A0044CC0C0046EE0E0048CA
:108A80001111004A3313004C9F14004E0B16005076
:108A900077170052E31800544F1A0056BB1B0058BA
:108AA000271D005ADD1D005C931E005E491F0060FB
:108AB00000200062B52000646C210066222200685C
:108AC000D822006A8E23006C4424006E000000341B
:108AD00000000036000000380000003A0000003CB2
:108AE0000000003E00000040000000420000004482
:108AF00000000046000000480000004A0000004C52
:108B00000000004E00000050000000520000005421
:108B100000000056000000580000005A0000005CF1
:108B20000000005E000000600000006200000064C1
:108B30000000006600000068441458585870111175
:108B40005858587041115858487011144858587066
:108B50001411584858703313005695130054B61327
:108B600000525A140050FD14004EA115004C451639
:108B7000004A761600486C17004672180044BA196D
:108B80000042741B0040911D003EB420003C9F2217
:108B9000003AE1220038532300368B24003481252B
:108BA00000322B2700302028002E5829002CB02A14
:108BB000002A9B2C0028D22D00267C2F0024263151
:108BC000002202330020FD34001E5C37001CCC3C28
:108BD000001A873E0018BE3F0016004000140040F7
:108BE0000012004000100040000E0040000C004049
:108BF000000A004000080040000600400004004059
:108C0000000200400000E8190056E8190054E81975
:108C10000052E8190050E819004EE819004CE81914
:108C2000004A1E1A00482C1B0046011D0044B51DB9
:108C300000429C1F0040EE21003EF923003C162616
:108C4000003A5E260038DC260036322800344129FE
:108C50000032152B0030242C002E7A2D002CF42EFF
:108C6000002A11310028683200263C3400241136D5
:108C700000221B3800204A3A001EE53C001C004040
:108C8000001A004000180040001600400014004088
:108C90000012004000100040000E0040000C004098
:108CA000000A0040000800400006004000040040A8
:108CB000000200400000000001020304050005005E
:108CC000010203040104000305020000F00100009A
:108CD00036010000F8000000BA0000007C0000002F
:108CE0007C0000007C000000411414111114441198
:108CF000141441110000290052007B00A400CC0094
:108D0000F5001E01470170019901C201EA01130239
:108D10003C0265028E02B602DF02080330035903EB
:108D20008203AA03D303FB0324044C0475049D04AB
:108D3000C504EE0416053E0567058F05B705DF057A
:108D400007062F0657067F06A706CE06F6061E075D
:108D500046076D079507BC07E4070B08320859085A
:108D60008108A808CF08F6081D0944096A09910975
:108D7000B809DE09050A2B0A520A780A9E0AC40AB3
:108D8000EA0A100B360B5C0B820BA80BCD0BF30B16
:108D9000180C3E0C630C880CAD0CD20CF70C1C0D9F
:108DA000410D650D8A0DAF0DD30DF70D1C0E400E54
:108DB000640E880EAC0ECF0EF30E170F3A0F5E0F37
:108DC000810FA40FC70FEA0F0D103010531075104C
:108DD0009810BA10DD10FF10211143116511871191
:108DE000A911CA11EC110D122E1250127112921209
:108DF000B312D412F41215133613561376139613B6
:108E0000B713D713F6131614361456147514941496
:108E1000B414D314F214111530154E156D158C15AC
:108E2000AA15C815E7150516231641165F167C16F8
:108E30009A16B716D516F2160F172C17491766177C
:108E40008317A017BC17D917F51711182E184A1831
:108E5000661881189D18B918D418F0180B1926191E
:108E600042195D1978199219AD19C819E219FD193D
:108E7000171A311A4C1A661A801A991AB31ACD1A8F
:108E8000E61A001B191B331B4C1B651B7E1B971B13
:108E9000AF1BC81BE11BF91B121C2A1C421C5A1CCD
:108EA000721C8A1CA21CBA1CD21CE91C011D181DB4
:108EB000301D471D5E1D751D8C1DA31DBA1DD01DC7
:108EC000E71DFD1D141E2A1E401E571E6D1E831E0B
:108ED000981EAE1EC41EDA1EEF1E051F1A1F2F1F7E
:108EE000451F5A1F6F1F841F991FAE1FC21FD71F18
:108EF000EC1F002000006400C9002D019201F70161
:108F00005B02C00224038903ED035204B6041A0570
:108F10007F05E3054706AB060F077307D7073B0836
:108F20009F0802096609C9092D0A900AF30A560B1F
:108F3000B90B1C0C7F0CE20C440DA60D090E6B0E38
:108F4000CD0E2F0F900FF20F5310B4101511761194
:108F5000D71138129812F8125813B813181477143E
:108F6000D61435159415F3155116B0160E176B1748
:108F7000C91726188318E0183D199919F519511ABF
:108F8000AD1A081B631BBE1B181C731CCD1C261DB1
:108F9000801DD91D321E8A1EE31E3B1F921FEA1F31
:108FA00041209820EE2044219A21EF214522992248
:108FB000EE2242239623E9233C248F24E224342505
:108FC0008525D72528267826C82618276827B72775
:108FD00006285428A228EF283D298929D629222AA3
:108FE0006D2AB82A032B4D2B972BE12B2A2C722CA0
:108FF000BB2C022D4A2D912DD72D1D2E632EA82E70
:10900000EC2E302F742FB82FFA2F3D307F30C03028
:10901000013141318131C13100323F327D32BA32CA
:10902000F73234337033AC33E73322345C34953465
:10903000CE3407353F357735AE35E4351A36503600
:109040008536B936ED36203753378637B737E937A7
:10905000193849387938A838D738053932395F395D
:109060008B39B739E2390D3A373A603A893AB23A30
:10907000DA3A013B283B4E3B733B983BBD3BE03B20
:10908000043C263C483C6A3C8B3CAB3CCB3CEA3C39
:10909000093D273D443D613D7D3D993DB43DCE3D7B
:1090A000E83D013E1A3E323E493E603E763E8C3EF1
:1090B000A13EB53EC93EDC3EEF3E013F123F233F9D
:1090C000333F433F513F603F6E3F7B3F873F933F7E
:1090D0009E3FA93FB33FBC3FC53FCD3FD53FDC3F9F
:1090E000E23FE83FED3FF13FF53FF93FFB3FFD3FFA
:1090F000FF3FFF3FFF3F0000E7382C35002020EF07
:109100002037202333202620210000800200040085
:10911000080010000002000400080400000200041F
:1091200000080010002000400080040000000080C3
:1091300000000040000000200000001000000008B7
:109140000000000400000002000000010000800098
:109150000000400000002000000010000000080097
:109160000000040000000200000001000080000078
:1091700000080140000C0140000C0140000C0140BF
:10918000000C0140000C0140000C0140000C0140AB
:10919000001001400010014000100140001001408B
:1091A000001001400010014000100140001001407B
:1091B0000014014004080140040C0140040C01406B
:1091C000040C0140040C0140040C0140040C01405B
:1091D000040C01400410014004100140041001403F
:1091E000041001400410014004100140041001402B
:1091F000041001400414014008080140080C01401B
:10920000080C0140080C0140080C0140080C01400A
:10921000080C0140080C01400810014008100140F2
:1092200008100140081001400810014008100140DA
:109230000810014008100140081401400C080140CA
:109240000C0C01400C0C01400C0C01400C0C0140BA
:109250000C0C01400C0C01400C0C01400C100140A6
:109260000C1001400C1001400C1001400C1001408A
:109270000C1001400C1001400C1001400C14014076
:1092800010080140100C0140100C0140100C01406E
:10929000100C0140100C0140100C0140100C01405A
:1092A000101001401010014010100140101001403A
:1092B000101001401010014010100140101001402A
:1092C0001014014000000000000000000000000039
:1092D000000000000000000014080140140C0140D0
:1092E000140C0140140C0140140C0140140C0140FA
:1092F000140C0140140C01401410014014100140E2
:1093000014100140141001401410014014100140C9
:10931000141001401410014014140140000000001A
:10932000000000000000000000000000000000003D
:10933000FFFFFF0F0FFFFFFFFFF0FFFFFF0FFFFF1C
:10934000FFFFF0FF0FFFFFFFFFF0FFFFFF0FFFFF2B
:10935000FFF0FFFF0FFFFFFFFFF0FFFFFF0FFFFF1B
:10936000FFFFF0FFFFFF0FFFFFFFFFF0FFFFFF0F0B
:10937000FFF0FFFF0000004040000000000400007C
:109380000040000000000400400000000004000055
:109390000040000000040000400000000004000045
:1093A0000040000000000400000040000000000435
:1093B0000000004000040000000000808000000069
:1093C000000800000080000000000800800000008D
:1093D000000800000080000000080000800000007D
:1093E000000800000080000000000800000080006D
:1093F00000000008000000800008000000000020BD
:109400002000000000020000002000000000020018
:109410002000000000020000002000000002000008
:1094200020000000000200000020000000000200F8
:1094300000002000000000020000002000020000E8
:1094400000000060600000000006000000600000F6
:109450000000060060000000000600000060000040
:109460000006000060000000000600000060000030
:109470000000060000006000000000060000006020
:109480000006000000800200040008001000000236
:10949000000400080400000200040008001000207E
:1094A0000040008004000000FF7FFFFFFDFFFFFF82
:1094B000FBFFFFFFF7FFFFFFEFFFFFFFFFFDFFFFDA
:1094C000FFFBFFFFFFF7FFFFFBFFFFFFFFFDFFFFBE
:1094D000FFFBFFFFFFF7FFFFFFEFFFFFFFDFFFFFD8
:1094E000FFBFFFFFFF7FFFFFFBFFFFFF0102030442
:1094F0000500020304050001030405000102050044
:109500000102030404050001020355050010AA1A14
:1095100055250030AA3A0000AA0A55150020AA2AAB
:109520005535FF3F4495000800000020200700004B
:10953000E80600083496000820070020C009000053
:10954000A464000845020406082D01020304040572
:10955000440607080913C12B1B08D5042113551510
:109560002A40061908019713093E1B082D041A29E1
:1095700004012D17020604050103148020FF8BAAA5
:109580000A02019C15AA0A551500085920AA2A5555
:1095900035FF3F072903010504060203127C1573FA
:1095A000FFFF04FF8080010125025B6402130A13A0
:1095B000116812081201100C0504060203010103D0
:1095C000070505280B010203040206070303040C28
:1095D0003D0706040509191F191904310506064B34
:1095E000AA1A024B381E026910312E40FD39692635
:1095F0000211042F405F020C26405B262ACD551530
:109600005515123902017F0316D0071AFF01013BDD
:109610000261AA6C080108A80916C491220312105D
:109620000A17401C12600A16901B01491325680294
:04963000000800002E
:020000040800F2
:10FC00004A46545A594D46312D4E3330202020203B
:10FC1000050406020301AA0AAA0AAA0AAA0AAA0A4B
:10FC2000AA0ADE3F00100000FF0131000201664613
:10FC300000400040513800400040004000400101B9
:10FC400000400040FF387B257B257B25FF003333B8
:10FC50000201401F00016626B81E6626FFFFFFFF57
:10FC6000FFFF01010100010000000300000200008D
:04FC70000000AA5591
:04000005080000ED02
:00000001FF
